:100000000C9463020C9480020C9480020C94800285
:100010000C9480020C9480020C9480020C94800258
:100020000C9480020C94280C0C9480020C94800296
:100030000C94D4180C9480020C9480020C94A01898
:100040000C9480020C9480020C94550B0C9480024A
:100050000C9464040C9480020C942E040C94800282
:100060000C945F0D0C9480020C9470170C94800219
:100070000C947C3D0C9480020C9480020A0A0D00C2
:100080004E65757472616C0048656164696E67489D
:100090006F6C64000A0D436F6E74726F6C3A2000CF
:1000A0004F4B0A0D000A0D43616C696272617469FD
:1000B0006E67206169722070726573737572652056
:1000C00073656E736F722E2E000A0D414343206ECE
:1000D0006F742063616C6962726174656421000AE7
:1000E0000D3D3D3D3D3D3D3D3D3D3D3D3D3D3D3D70
:1000F0003D3D3D3D3D3D3D3D3D3D3D3D3D3D3D006D
:100100000A0D466C69676874436F6E74726F6C0A8F
:100110000D48617264776172653A25642E25640A20
:100120000D536F6674776172653A5625642E2564A7
:10013000256320002E0048693A2534692020436653
:100140003A253469200047733A25346920205961E3
:100150003A25346920004E693A2534692020526FCF
:100160003A253469200045787465726E436F6E7469
:10017000726F6C20200052616E67653A2533692DDD
:1001800025336900506F736974696F6E3A202533A7
:100190006900536574706F696E742020253369009F
:1001A000536572766F202000506F343A20253369F2
:1001B00020506F383A2025336900506F333A20259C
:1001C000336920506F373A2025336900506F323A37
:1001D0002025336920506F363A2025336900506F4F
:1001E000313A2025336920506F353A202533690094
:1001F0004F6666436F757273653A2025356900480E
:10020000656164696E673A20202025356900436F77
:10021000757273653A2020202025356900436F6D83
:1002200070617373202020202020200052432D4C29
:100230006576656C3A2025356900566F6C74616788
:10024000653A20202535690048656967687420256E
:10025000346920282533692900526F6C6C202020D6
:10026000253469202825336929004E69636B2020D5
:100270002025346920282533692900414343202D56
:100280002053656E736F72005961772020253469A1
:10029000202825336929282533692900526F6C6C81
:1002A0002025346920282533692928253369290028
:1002B0004E69636B20253469202825336929282558
:1002C0003369290059617720202534692028253396
:1002D000692900526F6C6C20253469202825336908
:1002E00029004E69636B202534692028253369294C
:1002F0000059617720202534692028253369290099
:10030000526F6C6C20253469202825336929004EF2
:1003100069636B20253469202825336929004779D2
:10032000726F202D2053656E736F720050333A2523
:100330003469202050343A253469200050313A2560
:100340003469202050323A253469200047733A2519
:100350003469202059613A25346920004E693A25D4
:1003600034692020526F3A253469200043373A25FA
:100370003469202043383A253469200043353A2532
:100380003469202043363A253469200043333A2526
:100390003469202043343A253469200043313A251A
:1003A0003469202043323A2534692000486561646D
:1003B000696E673A20202025356900526F6C6C3ACF
:1003C000202020202020253569004E69636B3A20CB
:1003D00020202020202535690041747469747564DB
:1003E000650048656967687420436F6E74726F6C4E
:1003F000004E6F20004F6666736574202020203AFF
:10040000253569004169722050726573732E3A2553
:1004100035690053657420506F696E743A20253534
:1004200069004865696768743A202020202535698D
:100430000028632920486F6C6765722042757373CA
:100440000053657474696E673A202564200048572C
:100450003A5625642E25642053573A25642E256488
:100460002563002B204D696B726F4B6F7074657242
:10047000202B005B25695D005B25695D000A0D5539
:1004800073696E6720506172616D65746572205387
:100490006574202564000A0D496E69742E20454557
:1004A00050524F4D3A2047656E65726174696E67B0
:1004B0002044656661756C742D506172616D657460
:1004C00065722E2E2E0011241FBECFEFD0E1DEBFAD
:1004D000CDBF14E0A0E0B1E0E2E8F4E802C005908E
:1004E0000D92A43CB107D9F718E0A4ECB4E001C028
:1004F0001D92A83CB107E1F70E9482020C94404291
:100500000C940000CF93DF93F89414B815B8189B9F
:1005100006C0199B02C08DE003C08BE001C08AE0D9
:100520008093000184B1836084B9209100012A3056
:1005300011F4289A03C028982C3010F4299801C08F
:10054000299A84B7877F84BF8091600088618093F7
:1005500060001092600080ED97E09093E00480933B
:10056000DF04109274071092730710927D051092A9
:100570007C0510927B0510927A05109279051092F5
:1005800078052A3011F4289801C0289A0E94200B7F
:100590000E94050C0E940406809100018B3010F02F
:1005A0000E941F3D0E946C180E94420D0E9411176C
:1005B00078941092710686E48093720688E08093A6
:1005C000730681E08093740620910001822F6AE017
:1005D0000E947141492F50E0822F0E94714190E0AA
:1005E00024E630E03F932F9326E430E03F932F93AF
:1005F0001F921F925F934F939F938F9380E091E0A0
:100600009F938F931F920E947C088FED90E09F93A1
:100610008F931F920E947C088DB79EB740960FB6AD
:10062000F8949EBF0FBE8DBF809100018C3010F4F6
:10063000299A01C029980E94683C84E00E94123ADD
:100640008050944050F089EC90E09F938F931F92DC
:100650000E947C080F900F900F9084EF91E00E9411
:10066000B90BEC01CE010E94C20B8823D9F3809113
:10067000DF0780FF20C085EA90E09F938F931F9251
:100680000E947C0888EE93E00E94B90BEC010E9466
:10069000FB100F900F900F90CE010E94C20B882389
:1006A000D9F380EA90E09F938F931F920E947C0879
:1006B0000F900F900F900E947422809100018A3059
:1006C00011F4289801C0289A80ED97E09093E004F7
:1006D0008093DF0485E580937B0684E990E09F9317
:1006E0008F931F920E947C088091DF070F900F90DC
:1006F0000F9082FF03C088E890E002C080E890E09D
:100700009F938F931F920E947C080F900F900F90E1
:100710008CE790E09F938F931F920E947C080E9429
:100720003B1180ED97E090937503809374030F90D5
:100730000F900F908091DC048823E1F31092DC0489
:100740000E941F240E94C721209100012A3011F429
:10075000289801C0289A80910301882321F08150B4
:100760008093030112C01092D0041092D104109211
:100770008506109289051092880510928B051092BB
:100780008A0510928D0510928C05809174039091CA
:100790007503892B01F585E090E0909375038093B4
:1007A00074030E943E1780910403909105038F5FAC
:1007B0009F4FF9F48091670580FF1BC080E197E2AD
:1007C0009093E0048093DF0480E890E09093050329
:1007D000809304030EC08091740390917503019778
:1007E00090937503809374032A3011F4289801C004
:1007F000289A8091DC04882321F08091670580FD90
:1008000002C00E946B060E941307CE010E94C20B19
:10081000882309F120910C0330910D038091EF079B
:1008200090E02817390794F480E093E09093050353
:10083000809304038091DF049091E004892B31F4CC
:1008400080E797E19093E0048093DF0484E190E0F7
:100850000E94B90BEC010E94A0166CCF1F920F9260
:100860000FB60F9211248F939F93EF93FF93809174
:1008700002018823E1F48091D8049091D904019673
:100880009093D9048093D804FC01E853F94FE08198
:10089000ED3019F08639910539F41092D90410928F
:1008A000D80481E080930201E093C60004C0109256
:1008B000D9041092D804FF91EF919F918F910F90DE
:1008C0000FBE0F901F9018951F920F920FB60F92A8
:1008D00011242F933F934F935F936F937F938F9345
:1008E0009F93AF93BF93CF93DF93EF93FF93709159
:1008F000C6008091CA04882309F06DC06091D504B8
:10090000662371F4733279F47093D90581E0809392
:10091000D50483E290E09093D7048093D6045BC023
:10092000663908F054C0A62FB0E02091D60430916B
:10093000D7047D3069F0A752BA4F7C936F5F609304
:10094000D504270F311D3093D7042093D60443C01C
:10095000FD01E952FA4F9081ED01C852DA4F8881CA
:10096000A901491B5109481B51095F705093D704D5
:100970004093D6042081CA0136E0969587953A9532
:10098000E1F7835C8217F1F49881842F8F73835C85
:100990008917C1F481E08093CA046093CB04A75205
:1009A000BA4F7C938091DB05823571F488E190E049
:1009B0002CE00FB6F894A895809360000FBE2093AA
:1009C000600002C01092CA041092D50404C01092B4
:1009D000D5041092CA04FF91EF91DF91CF91BF919E
:1009E000AF919F918F917F916F915F914F913F91C7
:1009F0002F910F900FBE0F901F901895DC0140E0D3
:100A000050E020E030E008C0FA01E853F94F80815F
:100A1000280F311D4F5F5F4F4A175B07A9F73F70E3
:100A2000C90146E0969587954A95E1F7835CFD01FB
:100A3000E853F94F808311962F73235CFD01E8532F
:100A4000F94F2083A753B94F8DE08C931092020188
:100A50008091C8068093C60008951F93CF93DF93BB
:100A6000EA01722F93E29093C8066093C9068093BF
:100A7000CA06A3E0B0E060E04FC0FE01E60FF11D42
:100A800090816F5F715019F410E040E00FC0FE01DB
:100A9000E60FF11D40816F5F715011F410E006C048
:100AA000FE01E60FF11D10816F5F7150892F869551
:100AB0008695835CFD01E853F94F808350E09A01ED
:100AC00084E0369527958A95E1F7892F90E0837029
:100AD0009070F4E0880F991FFA95E1F7282B235CBA
:100AE000FD01E753F94F2083812F829586958695E6
:100AF00083704F705070440F551F440F551F842B47
:100B0000835CFD01E653F94F80831F73135CFD0185
:100B1000E553F94F10831496772309F0AECFCD013A
:100B20000E94FE04DF91CF911F9108950F931F93B0
:100B3000CF93DF93EC01062F70E0A22FB0E0129765
:100B40004AC0E42FF0E0E752FA4F30814F5FE42FC4
:100B5000F0E0E752FA4F50814F5FE42FF0E0E752A8
:100B6000FA4F10814F5FE42FF0E0E752FA4F2081F7
:100B70004F5F842F90E0A817B90784F1701771F1C7
:100B80005D53FE01E70FF11D852F82958F703D5358
:100B9000330F330F382B3083613001F1912F9D5388
:100BA0007F5FFE01E70FF11D71505295507F892F35
:100BB00086958695582B508363506F3F79F07E5F02
:100BC000FE01E70FF11D9295990F990F907C2D531F
:100BD000922B90837F5F662309F0B3CFDF91CF9193
:100BE0001F910F9108951F93182F8A3019F48DE0EB
:100BF0000E94F3058091C00085FFFCCF1093C600D2
:100C000080E090E01F9108951F931FB7F8948091A2
:100C1000C1008F778093C1008091C1008F7B80934A
:100C2000C100589A5098599A519A1092C5008AE278
:100C30008093C4008091C00082608093C00088E1EE
:100C40008093C1008091C2008F778093C200809111
:100C5000C2008F7B8093C2008091C2008F7D809301
:100C6000C2008091C2008F7E8093C2008091C2003A
:100C7000877F8093C2008091C1008B7F8093C100E9
:100C80008091C20084608093C2008091C200826023
:100C90008093C20002C08091C6008091C00087FD91
:100CA000FACF8091C10080688093C1008091C1001B
:100CB00080648093C1001092CA0481E08093020195
:100CC00088EC90E00E94B90B9093700680936F06B9
:100CD0001FBF1F91089580910201882309F4A2C0CB
:100CE0008091C504882371F080910201882351F01E
:100CF0006091D4042BE04BE756E087E40E942D0579
:100D00001092C50480916F06909170060E94C20BEC
:100D1000882321F48091C7048823B1F080910201D7
:100D2000882391F06091D40422E446E856E084E4FC
:100D30000E942D051092C7048AEF90E00E94B90B23
:100D40009093700680936F06609101016F3F89F068
:100D5000462F50E094E0440F551F9A95E1F74C5F01
:100D60005E4F605D20E181E40E942D058FEF80934E
:100D7000010190915E079923A1F0809102018823DF
:100D800081F083E28093C8069093C9068DE080933A
:100D9000CA061092020110925E078091C8068093E5
:100DA000C6008091C604882359F1809102018823EE
:100DB00039F10E9444111092C6043091C904932F56
:100DC0009F5F9093C904943021F08091C8048823D8
:100DD00059F02EE14FE657E060E084E30E942D05D4
:100DE0008FEF8093C9040CC044E1949FA0011124AB
:100DF0004F5D5C4F24E160E0832F8F5C0E942D05E6
:100E00008091C404882371F080910201882351F0FD
:100E10006091D4042AE041E756E086E50E942D0562
:100E20001092C40408951F93CF93DF93CDB7DEB71C
:100E300022970FB6F894DEBF0FBECDBF8091CA04D3
:100E4000882309F4F6C08091DB058B3609F47FC056
:100E50008C3690F4833609F43FC0843630F4813602
:100E6000C1F0823609F0E3C020C0873609F47EC0A5
:100E7000883609F0DCC047C0813709F47BC0813770
:100E800008F4A2C0843709F459C0863709F0CFC0EE
:100E900069C02091CB0443E062E0CE0101960E943C
:100EA000960589818093010113C02091CB0443E012
:100EB0006BE08BE796E00E94960580910505909186
:100EC0007D06892B809305058091840680935E07BB
:100ED0008FEF80930301ABC02091CB0443E06BE024
:100EE0008BE796E00E9496058091050590917D061E
:100EF000892B809305058091840680935E0781E0AD
:100F00008093C704E5CF2091CB0443E062E0CE019B
:100F100001960E949605809105059981892B809301
:100F200005058A818F3F21F481E08093C80402C0C7
:100F30001092C80481E08093C60479C02091CB044C
:100F400043E064E08CEC94E00E949605C1CF2091D0
:100F5000CB0443E064E080ED94E00E94960580912C
:100F6000D304B4CF81E08093C40461C081E0809356
:100F7000C5045DC02091CB0443E062E0CE01019640
:100F80000E949605809102018823E1F389818F3FB9
:100F900071F0863010F085E0898389810E94423AA1
:100FA0006091D404898123E547ED57E009C0109191
:100FB000D40482E00E94013A23E547ED57E0612F17
:100FC000855B0E942D0533C02091CB0443E063E58F
:100FD00087ED97E00E9496058091DB058B560E9475
:100FE0002B3A6091020870E080E090E024EC39E058
:100FF00040E050E00E94524160937D0370937E0375
:1010000080937F03909380036091030870E080E0F9
:1010100090E00E9452416093810370938203809319
:101020008303909384030E94593C0E94DA23109218
:10103000CA0422960FB6F894DEBF0FBECDBFDF9173
:10104000CF911F910895982F80915F07813069F4A7
:1010500080910405E82FF0E0EF5DFC4F90838F5FF7
:101060008093040521E030E005C0892F0E94F3053C
:10107000282F30E0C90108951F93182F04C080E382
:101080000E94230811501116D4F31F9108951F9345
:10109000182F04C080E20E94230811501116D4F3C7
:1010A0001F9108950F931F93CF93DF938C01EB0152
:1010B00008C0F8010F5F1F4FE4918E2F0E94230894
:1010C00021972097B1F7DF91CF911F910F9108954C
:1010D0000F931F93CF93DF938C01EB0106C0F801B0
:1010E00081918F010E94230821972097C1F7DF91FA
:1010F000CF911F910F9108952F923F924F925F923F
:101100006F927F928F929F92AF92BF92CF92DF9217
:10111000EF92FF920F931F93CF93DF93CDB7DEB77C
:10112000E5970FB6F894DEBF0FBECDBF2B968FADFF
:101130002B9780935F07CE01835B9F4F9B838A83AE
:101140002D964EAC5FAC2D971EA61FA618AA19AA05
:101150009E01225D3F4F3DAB2CAB820102C00F5F71
:101160001F4FF801F490FF2019F0F5E2FF16B9F7D0
:10117000B8016419750919F0C2010E945208FF20D4
:1011800009F445C228010894411C511C1982AA8106
:10119000BB8133241BAA2FEF2AABF2010894411C18
:1011A000511CB490632D70E06170707035E7B31618
:1011B00021F08B2D80628837C9F46115710559F0D3
:1011C0002D913D914D915C9113972EA73FA748AB70
:1011D00059AB14960BC08D919C9111979C0140E0E6
:1011E00050E02EA73FA748AB59AB129630E2B3169A
:1011F00021F48981882389F61CC043E2B41611F4D6
:1012000058E055C08AE2B81621F09DE2B91671F493
:1012100008C0FD011296E081EBABE7FFBECFE19580
:10122000EBABE0E13E2AFFED3F22B7CF2BE2B21657
:1012300011F4B982B2CF3EE2B31699F5F2010894E7
:10124000411C511C84918A3221F0B82E20E030E0FC
:101250001DC0FD0112964081518157FF02C04FEF22
:101260005FEF4AAB9ACFC90153E0880F991F5A9597
:10127000E1F7220F331F280F391F2B0D311D20538B
:101280003040F2010894411C511CB4908B2D8053C6
:101290008A3048F3A90137FF02C04FEF5FEF4AAB36
:1012A00085CF40E3B41629F434FC77CF50E2352AD9
:1012B00074CF8B2D81538930D8F420E030E0C90100
:1012C00003E0880F991F0A95E1F7220F331F280FBB
:1012D000391F2B0D311D20533040F2010894411C61
:1012E000511CB4908B2D80538A3048F32BAB5ECFCA
:1012F00088E6B81619F494E0392A4FCFECE6BE160A
:1013000019F4F1E03F2A49CFBB83AA8323E6B21642
:1013100039F41296BB83AA8312978C918E8322C1D3
:1013200034E4B31639F044E6B41631F059E6B51694
:10133000A9F502C081E0382A30FE08C01496BB83AC
:10134000AA835E914E913E912E910AC01296BB8364
:10135000AA839E918E919C01442737FD4095542F7E
:101360002EA73FA748AB59AB8EA59FA5A8A9B9A9A1
:10137000BB238CF42EA53FA548A959A950954095AB
:10138000309521953F4F4F4F5F4F2EA73FA748AB5A
:1013900059AB8DE28983BAE02B2E80C03FE4B316AF
:1013A00021F04FE6B41631F402C051E0352AA8E02E
:1013B0002A2E73C080E7B81689F41296BB83AA83DD
:1013C0009E918E919C0140E050E02EA73FA748AB34
:1013D00059AB30E4332AF8E7BF2E5DC043E7B416BB
:1013E000D1F51296BB83AA83DE90CE90C114D104AE
:1013F00089F488E28E838EE68F8385E788878CE682
:1014000089878A8789E28B871C86E6E0CE2ED12CDD
:10141000CC0EDD1E5AA957FD14C0452F552747FD98
:10142000509560E070E0C6010E942A3F009711F4D9
:10143000FAA80EC0F82EFC188AA98F154CF4F82EC5
:1014400007C0F60101900020E9F73197FE2EFC1845
:10145000198240E090C095E5B91621F0A5E7BA16CB
:1014600031F402C0B1E03B2A7AE0272E16C0E8E54D
:10147000BE1621F0F8E7BF1609F070C033FE0BC0AE
:101480002EA53FA548A959A92115310541055105AA
:1014900011F030E4332A60E1262E19824AA947FD73
:1014A00002C05FED35228EA59FA5A8A9B9A9009716
:1014B000A105B10549F49AA9992331F45EE2C52E3C
:1014C000D12CCC0EDD1E46C06EA47FA488A899A89E
:1014D0004EE2C42ED12CCC0EDD1EE22CFF2400E007
:1014E00010E06EA57FA588A999A9A80197010E947F
:1014F000A4416A3020F430E3A32EA60E08C027E5ED
:10150000A22EA60EA8E5BA1611F4BFEDAB22F60185
:10151000A2926F016EA57FA588A999A9A80197013C
:101520000E94A4412EA73FA748AB59AB6E147F047D
:101530008006910618F039014A01D3CFF8E02F1642
:1015400049F433FE07C020E3A21621F080E3D60160
:101550008E936D01FCA8FC184AA90DC0BB2009F4AC
:1015600056C0BE82198296E0C92ED12CCC0EDD1E4B
:1015700040E0FF24F394E42EEF18E7FCEE24898189
:10158000882319F08F2D8F5F06C036FC02C08F2D87
:1015900002C08F2D8E5FA82EAE0C032D10E080E3CD
:1015A000882E912C802291228114910421F48BA900
:1015B0008A190E9447088981882329F061E070E038
:1015C000CE01019609C006FF09C080E38C83BD826D
:1015D00062E070E0CE0104960E946808B0E28B16CB
:1015E000910421F48BA98A190E943C088E2D0E9437
:1015F0003C086F2D772767FD7095C6010E9468082B
:1016000004FFABCD8BA98A190E944708A6CDE596A9
:101610000FB6F894DEBF0FBECDBFDF91CF911F9103
:101620000F91FF90EF90DF90CF90BF90AF909F9081
:101630008F907F906F905F904F903F902F90089584
:101640002FB7F894909100019A3019F4529A5A9851
:1016500002C03F9A479884B1886184B985B1877E7A
:1016600085B99A3019F4529A5A9802C03F9A47980D
:1016700084B58F7A84BD84B5836A84BD85B587734C
:1016800085BD85B5887F826085BD17BC88E788BD2C
:1016900016BC80916E00897F80936E0080916E00F1
:1016A000816080936E002FBF08951F920F920FB636
:1016B0000F9211242F933F938F939F938091E10476
:1016C00081508093E1048F3FB9F489E08093E10475
:1016D000809106038F5F817080930603882319F43D
:1016E00081E08093DC048091DA049091DB04019620
:1016F0009093DB048093DA048091DF049091E004FE
:10170000892BB1F08091DF049091E00401979093D0
:10171000E0048093DF042091DF043091E0048091A5
:1017200004039091050382239323892BA1F406C01F
:101730008FEF9FEF90930503809304038091000146
:101740008A3039F404C05A9A0BC0479A09C05A9893
:1017500007C0479805C0809100018A30B1F7F3CFE8
:101760009F918F913F912F910F900FBE0F901F90DF
:1017700018952091DA043091DB0421503040820F1B
:10178000931F08952091DA043091DB04821B930BA0
:10179000892F99278078992787FD90950895AC0126
:1017A0002091DA043091DB042150304005C0809153
:1017B0007A00886C80937A008091DA049091DB043F
:1017C000B901681B790BCB01840F951F807090784D
:1017D000892F9927882359F30895AC012091DA04C1
:1017E0003091DB04215030408091DA049091DB0489
:1017F000B901681B790BCB01840F951F807090781D
:10180000892F9927882381F308959FB7F894579AD1
:101810005F98E0EBF0E080818F708083808183604F
:101820008083E1EBF0E08081847380838081846039
:1018300080831092B2008AE08093B300E0E7F0E08A
:1018400080818A7F80838081826080839FBF0895AA
:101850001F920F920FB60F9211240F931F932F9385
:101860003F934F935F936F937F938F939F93AF9328
:10187000BF93EF93FF938091070390910803843007
:10188000910520F4019708F0ADC0D1C0049709F08C
:10189000DDC080E390E09093E3048093E204209124
:1018A0009C0330E0220F331F4091090350910A033B
:1018B000CA01880F991F840F951F280F391F36956D
:1018C00027953695279530930A0320930903809135
:1018D000E2049091E304280F391F3093E30420932E
:1018E000E204809119086091F90720912705309151
:1018F00028054091290550912A0580FF12C00091CA
:10190000E2041091E30470E080E090E00E94524114
:1019100020E030E440E050E00E94C641020F131F77
:1019200011C00091E2041091E30470E080E090E0C7
:101930000E94524120E030E440E050E00E94C64165
:10194000021B130B1093E3040093E2048091E20462
:101950009091E3042091FA0743E0249F9001112421
:101960008217930728F43093E3042093E20410C015
:101970002091E2043091E3048091FB07849FC00131
:1019800011248217930720F49093E3048093E204D8
:101990008091E2049091E3049093B1068093B006A5
:1019A0008091E2049091E3046FEF70E00E947D412A
:1019B0008D9760F48091E2049091E304835B9F4FE4
:1019C0009093E3048093E20483E101C080E6809376
:1019D0000B038091E2049091E30480958093B3001F
:1019E00083EC32C08091E2049091E3048F3F910533
:1019F00081F078F05F9A83E08093B0008091E204F8
:101A00009091E3048F5F90409093E3048093E2040D
:101A10001DC083E88093B00080910B038093B300D6
:101A200081E090E090930803809307030FC08091BA
:101A3000FC0790E0880F991F880F991F9093080367
:101A4000809307035F9883E08093B0008091070341
:101A50009091080301979093080380930703FF91E7
:101A6000EF91BF91AF919F918F917F916F915F9116
:101A70004F913F912F911F910F910F900FBE0F909B
:101A80001F9018959FB7F89411B812B88FEF8093F4
:101A90007E00ECE7F0E080818F7180838081807E22
:101AA0008083AAE7B0E087E28C93EBE7F0E08081E7
:101AB000887F80838C91886C8C939FBF08951F9240
:101AC0000F920FB60F921124EF92FF920F931F9374
:101AD0002F933F934F935F936F937F938F939F9336
:101AE000AF93BF93CF93DF93EF93FF9380917A00EF
:101AF000877380937A00809102058F5F809302053F
:101B00008150853009F47EC0863090F4823009F42B
:101B100040C0833030F48823F1F0813009F084C272
:101B20002FC0833009F441C0843009F07DC25AC00F
:101B3000883009F4B2C0893038F4863009F473C0B3
:101B4000873009F071C28CC0893009F4C3C08A3073
:101B500009F06AC2DBC1809178009091790090937E
:101B600001058093000581E0809303058091F804CE
:101B70009091F90401969093F9048093F80458C267
:101B800080917800909179009093FF048093FE04F7
:101B900082C080917800909179009093FD048093A9
:101BA000FC0484E08093030543C240910C035091F0
:101BB0000D0380917800909179009A01220F331FD4
:101BC000240F351F63E070E00E947D41260F371F10
:101BD000369527953695279530930D0320930C0362
:101BE00086E0E0CF80912105909122052091780038
:101BF00030917900821B930B9093F0048093EF0453
:101C000087E0D0CF809178009091790020911F05D6
:101C100030912005821B930B9093F2048093F10482
:101C20001092030505C280910001209100053091BA
:101C300001058A3049F48091780090917900820FF3
:101C4000931F9695879506C08091780090917900B2
:101C5000820F931F9093EB048093EA0481E0A2CF5C
:101C6000809100012091FE043091FF048A3049F4F4
:101C70008091780090917900820F931F96958795B7
:101C800006C08091780090917900820F931F909305
:101C9000E9048093E80482E085CF809100012091DF
:101CA000FC043091FD048A3049F4809178009091D1
:101CB0007900820F931F9695879506C080917800D2
:101CC00090917900820F931F9093E7048093E6042C
:101CD00085E068CF6091780070917900E0902305ED
:101CE000F09024050091250510912605882777FDA1
:101CF0008095982F0E943740A80197010E94373F96
:101D00000E9404407093F4046093F304E091F304A0
:101D1000F091F4048091F1049091F204C091EF04E9
:101D2000D091F00497FF03C0909581959F4F64E098
:101D300070E00E9491419B01CE01D7FF03C09095B6
:101D400081959F4F64E070E00E949141260F371FFC
:101D5000E20FF31FF093F404E093F3048091F30493
:101D60009091F40402970CF43EC0609123057091A9
:101D70002405809125059091260520E030E84BE36D
:101D800054E40E94724088230CF078C060912305CF
:101D90007091240580912505909126052AE037ED64
:101DA00043EA5CE30E94383F609323057093240567
:101DB0008093250590932605809165059091660591
:101DC000845F914008F05AC060912305709124050A
:101DD00080912505909126052DEC3CEC4CEC5DE3C3
:101DE0000E94383F43C08091F3049091F4048F5FC8
:101DF0009F4F0CF043C060912305709124058091A2
:101E000025059091260520E030E849E054E40E9441
:101E1000764018169CF560912305709124058091F9
:101E20002505909126052AE037ED43EA5CE30E9400
:101E3000373F609323057093240580932505909385
:101E400026058091650590916605845F9140B0F408
:101E500060912305709124058091250590912605B8
:101E60002DEC3CEC4CEC5DE30E94373F6093230586
:101E70007093240580932505909326058091780022
:101E8000909179009093E5048093E40420915705A4
:101E9000309158054091590550915A058091F304AD
:101EA0009091F404AA2797FDA095BA2F820F931F53
:101EB000A41FB51F8093570590935805A09359050B
:101EC000B0935A05E0905705F090580500915905D8
:101ED00010915A05609157057091580580915905E8
:101EE00090915A0520E034E040E050E00E94C64165
:101EF000E21AF30A040B150BE0925705F09258050D
:101F00000093590510935A0583E04CCEE091780078
:101F1000F09179008091FA049091FB04E80FF91F89
:101F2000F093FB04E093FA048091F5048F5F8093B3
:101F3000F5048091F504853008F476C0809178002E
:101F40009091790090931603809315034091F604C5
:101F50005091F70420916007309161072E1B3F0BD1
:101F600080918E0590918F05281B390B80918B03F2
:101F700090E0BC01269FC001279F900D369F900DD9
:101F800011249A01A3E0220F331FAA95E1F7241B25
:101F9000350B820F931F68E070E00E9491417093AF
:101FA000F7046093F604E0901103F090120300919F
:101FB000130310911403BF01882777FD8095982F94
:101FC000A8019701220F331F441F551F2E0D3F1DDF
:101FD000401F511F620F731F841F951F24E030E0C4
:101FE00040E050E00E94C641209311033093120359
:101FF00040931303509314032091600730916107BD
:102000008091110390911203A0911303B0911403D6
:10201000281B390B30938F0520938E051092F50401
:102020001092FB041092FA0410920305109202051C
:1020300080917C00807E90910305892B80937C00A9
:1020400080910205882329F080917A00886C809322
:102050007A00FF91EF91DF91CF91BF91AF919F9166
:102060008F917F916F915F914F913F912F911F9130
:102070000F91FF90EF900F900FBE0F901F9018954B
:102080000F931F931092EC041092ED041092EE0443
:102090000CE810E0133019F40B3008F009E08091DF
:1020A000E6049091E7048C5F934024F480910E0342
:1020B00081500CC08091E6049091E70487509440D1
:1020C00014F411E006C080910E038F5F80930E031D
:1020D00010E08091E8049091E9048C5F934024F42F
:1020E00080910F0381500AC08091E8049091E90427
:1020F0008750944034F080910F038F5F80930F03DB
:1021000001C01F5F8091EA049091EB048C5F9340C3
:1021100024F48091100381500AC08091EA049091C8
:10212000EB048750944034F0809110038F5F8093CC
:10213000100301C01F5F87E080930A050E942817E3
:1021400080910E038A3030F481E08093EC048AE0C1
:1021500080930E0380910E03863F30F081E08093E0
:10216000EC0485EF80930E0380910F038A3030F4E6
:1021700081E08093ED048AE080930F0380910F0348
:10218000863F30F081E08093ED0485EF80930F036C
:10219000809110038A3030F481E08093EE048AE06D
:1021A0008093100380911003863F30F081E080938C
:1021B000EE0485EF8093100380910A058823E1F7F0
:1021C0001092F50480917A00886C80937A00809157
:1021D000F5048823E1F30A3020F48AE090E00E94BD
:1021E000CF0B015009F056CF86E490E00E94CF0B50
:1021F0001F910F9108951F93CF93DF9383E00E9467
:10220000013A182F853108F01A5017BD84E690E086
:102210000E94CF0B80911503909116038255934035
:10222000C0F410E016C017BD82E390E00E94CF0B0F
:10223000DF93CF931F920E947C08809115039091A9
:1022400016030F900F900F908458934030F01F5F4B
:1022500002C0C4E3D1E01A3F30F3612F83E00E9453
:102260000A3A109362078CE291E00E94CF0BDF9153
:10227000CF911F910895E1E2F3E080E2819383E042
:10228000E137F807D1F708951F9380910505282FAE
:1022900030E0C90181709070682F8823A9F0809187
:1022A0000605882311F0815002C08091710380934C
:1022B0000605E1E2F3E080E2819343E0E137F407D1
:1022C000D1F78FEF8093C904A9014270507021FFAC
:1022D00017C09091060580917103981719F4109218
:1022E000060503C09F5F90930605E1E2F3E080E2FC
:1022F000819383E0E137F807D1F78FEF8093C9042A
:10230000662321F0452B11F01092060580910605F9
:10231000282F30E08A3040F481E1809304053F9318
:102320002F9388E794E007C080E1809304053F93F2
:102330002F9383E794E09F938F9381E08F930E9484
:102340007C080F900F900F900F900F901091060542
:10235000153009F405C2163090F4123009F4D1C0DA
:10236000133030F4112309F1113009F0D1C465C0E4
:10237000133009F41CC1143009F0CAC475C11830F7
:1023800009F492C3193038F4163009F411C3173028
:1023900009F0BEC464C31A3009F421C41A3008F429
:1023A000C2C31B3009F0B4C45CC41092040583E6B8
:1023B00094E09F938F9311E01F930E947C0884E127
:1023C0008093040520910001822F6AE00E947141F0
:1023D000492F50E0822F0E94714190E024E630E0C6
:1023E0003F932F9326E430E03F932F931F921F9249
:1023F0005F934F939F938F938EE494E09F938F937B
:102400001F930E947C0888E2809304050E94593C37
:1024100090E09F938F9381E494E09F938F931F9319
:102420000E947C088CE38093040581E394E09F93F1
:102430008F931F930E947C080DC38091DF0780FF5C
:1024400042C01092040580918E0590918F059F9354
:102450008F9382E294E09F938F931F930E947C0856
:1024600084E18093040580919005909191059F935C
:102470008F9383E194E09F938F931F930E947C0836
:1024800088E28093040580911503909116039F9331
:102490008F9384E094E09F938F931F930E947C0816
:1024A0008CE3809304058091620790E09F938F9363
:1024B00085EF93E09F938F931F930E947C088DB7C5
:1024C0009EB744961FC484E18093040581EF93E096
:1024D0009F938F931F930E947C0888E2809304054A
:1024E00082EE93E09F938F931F930E947C084DB7D9
:1024F0005EB74A5F5F4F0FB6F8945EBF0FBE4DBF29
:102500000CC41092040589ED93E09F938F9311E022
:102510001F930E947C0884E1809304056091270545
:10252000709128058091290590912A0520E034E0DA
:1025300040E050E00E94C6415F934F933F932F933A
:102540008AEC93E09F938F931F930E947C0888E20C
:102550008093040560912F057091300580913105BD
:102560009091320520E034E040E050E00E94C64106
:102570005F934F933F932F938BEB93E09F938F93B6
:102580001F930E947C088CE380930405809177035D
:10259000909178039F938F938CEA93E09F938F930E
:1025A0001F930E947C088DB79EB74696ABC31092CE
:1025B0000405809173079091740720917107309101
:1025C00072079F938F933F932F938CE993E09F9390
:1025D0008F9311E01F930E947C0884E1809304058F
:1025E0008091770790917807209175073091760751
:1025F0009F938F933F932F938CE893E09F938F93B8
:102600001F930E947C0888E28093040580917B07D9
:1026100090917C072091790730917A079F938F934F
:102620003F932F938CE793E09F938F931F930E9488
:102630007C088CE38093040580917F07909180074C
:1026400020917D0730917E079F938F933F932F9327
:102650008CE693E09F938F931F930E947C084DB765
:102660005EB7445E5F4F47CF10920405E091D807F4
:10267000F0E0EE0FFF1FE159F84F20813181E0912A
:10268000D707F0E0EE0FFF1FE159F84F80819181ED
:102690003F932F939F938F938CE593E09F938F931A
:1026A00011E01F930E947C0884E180930405E0916F
:1026B000DA07F0E0EE0FFF1FE159F84F208131817A
:1026C000E091D907F0E0EE0FFF1FE159F84F80814C
:1026D00091813F932F939F938F938CE493E09F93EB
:1026E0008F931F930E947C0888E280930405E091F9
:1026F000DC07F0E0EE0FFF1FE159F84F2081318138
:10270000E091DB07F0E0EE0FFF1FE159F84F808109
:1027100091813F932F939F938F938CE393E09F93AB
:102720008F931F930E947C088CE380930405E091B3
:10273000DE07F0E0EE0FFF1FE159F84F20813181F5
:10274000E091DD07F0E0EE0FFF1FE159F84F8081C7
:1027500091813F932F939F938F938CE293E036C2A6
:10276000109204058EE193E09F938F9311E01F93E5
:102770000E947C080F900F900F90809100018A308A
:1027800021F08B3009F0AAC04DC084E1809304058C
:1027900020911505309116058091E6049091E7048B
:1027A000821B930B3F932F939F938F938FE093E024
:1027B0009F938F931F930E947C0888E28093040567
:1027C00020911705309118058091E8049091E90453
:1027D000821B930B3F932F939F938F9380E093E003
:1027E0009F938F931F930E947C088CE38093040532
:1027F0002091190530911A058091EA049091EB041B
:10280000A901481B590B3F932F935F934F9381EF7F
:1028100092E09F938F931F930E947C088DB79EB781
:10282000459670C284E1809304052091150530918E
:102830001605C90162E070E00E9491418091E604B2
:102840009091E704821B930B7F936F939F938F93D9
:1028500082EE92E09F938F931F930E947C0888E200
:10286000809304052091170530911805C90162E095
:1028700070E00E9491418091E8049091E904821BEC
:10288000930B7F936F939F938F9383ED92E09F932E
:102890008F931F930E947C088CE380930405209102
:1028A000190530911A05C90162E070E00E9491415A
:1028B0008091EA049091EB04281B390B7F936F936E
:1028C0003F932F9384EC92E09F938F931F930E94EA
:1028D0007C084DB75EB74B5E5F4F0DCE84E18093B1
:1028E000040520910E0330E0E0911505F0911605E6
:1028F000CF0162E070E00E9491418091E6049091E6
:10290000E7048E1B9F0B3F932F937F936F939F93AF
:102910008F9380EB92E09F938F931F930E947C088C
:1029200088E28093040520910F0330E0E0911705C1
:10293000F0911805CF0162E070E00E949141809112
:10294000E8049091E9048E1B9F0B3F932F937F9394
:102950006F939F938F938CE992E09F938F931F9334
:102960000E947C088CE380930405E0911003F0E062
:102970002091190530911A05C90162E070E00E94AA
:1029800091418091EA049091EB04281B390BFF934D
:10299000EF937F936F933F932F9388E892E09F93F9
:1029A0008F931F930E947C088DB79EB74B96AAC148
:1029B000109204058BE792E09F938F9311E01F9391
:1029C0000E947C0884E18093040580911F0590910A
:1029D00020052091F1043091F2049F938F933F934F
:1029E0002F938AE692E09F938F931F930E947C0817
:1029F00088E2809304058091210590912205209121
:102A0000EF043091F0049F938F933F932F9389E5C8
:102A100092E09F938F931F930E947C088CE3809396
:102A200004056091230570912405809125059091FE
:102A300026050E9404402091BA073091BB077F937E
:102A40006F933F932F9388E492E09F938F931F930C
:102A50000E947C084DB75EB7485E5F4F4CCD84E165
:102A60008093040580910C0390910D039F938F93A5
:102A70008AE392E09F938F9311E01F930E947C085A
:102A800088E28093040580910E0590910F059F9335
:102A90008F938CE292E09F938F931F930E947C0808
:102AA0008DB79EB70A962EC1109204058DE192E073
:102AB0009F938F9311E01F930E947C0884E1809381
:102AC00004058091790390917A039F938F938EE010
:102AD00092E09F938F931F930E947C0888E28093DB
:102AE000040580917703909178039F938F938FEFE4
:102AF00091E09F938F931F930E947C088CE38093B7
:102B0000040580915B0590915C059F938F9380EF06
:102B100091E09F938F931F930E947C084DB75EB7FF
:102B20004E5E5F4FE8CC1092040580917005909145
:102B3000710520916805309169059F938F933F93AC
:102B40002F938EED91E09F938F9311E01F930E943E
:102B50007C0884E18093040580917205909173054F
:102B600020916A0530916B059F938F933F932F932C
:102B70008CEC91E09F938F931F930E947C0888E2D6
:102B800080930405809174059091750520916C05E2
:102B900030916D059F938F933F932F938AEB91E034
:102BA0009F938F931F930E947C088CE3809304056E
:102BB000809176059091770520916E0530916F0593
:102BC0009F938F933F932F9388EA91E09F938F93E6
:102BD0001F930E947C088DB79EB74C9693C01092AD
:102BE000040580EA91E09F938F9311E01F930E9468
:102BF0007C0884E18093040580919C0390E09F937E
:102C00008F9382E991E09F938F931F930E947C089A
:102C100088E2809304058091E2049091E3049F93FD
:102C20008F9384E891E09F938F931F930E947C0879
:102C30008CE3809304052091FB0730E08091FA0734
:102C400090E03F932F939F938F9386E791E09F931C
:102C50008F931F930E947C084DB75EB74C5E5F4F09
:102C60004ACC1092040586E691E09F938F9311E081
:102C70001F930E947C0884E18093040520917F06C5
:102C8000332727FD309580917E06992787FD909503
:102C90003F932F939F938F9386E591E09F938F931C
:102CA0001F930E947C0888E280930405209180068F
:102CB000332727FD30958091810690E03F932F9335
:102CC0009F938F9386E491E09F938F931F930E942D
:102CD0007C088CE3809304052091850630E0809188
:102CE0008206992787FD90953F932F939F938F930B
:102CF00086E391E09F938F931F930E947C088DB78A
:102D00009EB748960FB6F8949EBF0FBE8DBF05C004
:102D100011501093710310920605109205051F9132
:102D2000089587B18C6087B942984398109207053F
:102D300080E88093720310920805809373030895CE
:102D4000809109058150809309058F3F09F068C083
:102D500084E08093090580910C088B3F80F080917E
:102D6000A203873E28F080910B0888231CF124C021
:102D70008A3028F480910B088823F4F01BC08091DE
:102D800007058150809307058F3FB9F48091A20316
:102D900081508093070580917203813011F480E89F
:102DA00001C086958093720380910B089091720305
:102DB000892311F0429A01C0429880910E088B3FFE
:102DC00088F08091A303873E28F080910D08882326
:102DD00024F106C08A3030F480910D0887FF1DC0B1
:102DE00043980895809108058150809308058F3F8E
:102DF000B9F48091A30381508093080580917303F7
:102E0000813011F480E801C086958093730380912E
:102E10000D0890917303892311F0439A0895439804
:102E200008959FB7F8943998389A88B1836088B923
:102E3000E9EBF0E080818C7F80838AE28093B800A8
:102E400010920A0510920B0510920C059FBF089571
:102E500085EA8093BC00089584E98093BC000895BE
:102E60008093BB0085E88093BC00089585EC809337
:102E7000BC00089585E88093BC000895EF92FF920E
:102E80000F931F938CEBE82EF12C84E9F7018083DC
:102E900010920A050BEB10E0F801808180930B057E
:102EA00010920B0510920C0580E8F70180831092B8
:102EB000BD001092BA00F80110821092B900109271
:102EC000B8000E94111785EAF7018083F80110828B
:102ED00085E8F70180831F910F91FF90EF9008958F
:102EE0001F920F920FB60F9211248F939F93EF931F
:102EF000FF9380910A058F5F80930A05815085308A
:102F000009F471C0863090F4823009F453C08330E4
:102F100030F4882309F1813009F0C6C022C0833023
:102F200009F45AC0843009F0BFC05BC0883009F48E
:102F300084C0893038F4863009F45EC0873009F0E7
:102F4000B3C079C08A3009F48FC08A3008F47AC0DF
:102F50008B3009F0A9C08AC080910B05880F8E5A6A
:102F600016C080910B058230C9F0833030F488237D
:102F700061F0813009F0A7C00EC08430A9F0843020
:102F800080F0853009F09FC012C08091C607809301
:102F9000BB0085E881C08091B107F9CF8091BC0763
:102FA000F6CF8091CF07F3CF8091BD07F0CF80910E
:102FB000D607EDCF84E98093BC0080910B05853066
:102FC00040F480910B058F5F80930B0510920A05EA
:102FD00062C010920B055FC080910C05880F8D5A5E
:102FE000D6CF85EC59C0E0910C05F0E08091BB0094
:102FF000ED59F84F8083CDCFE0910C05F0E0809142
:10300000BB00E959F84F808380910C058F5F809356
:103010000C0580910C05863010F010920C0584E9A7
:103020008093BC0010920A058AE090E090937503AB
:103030008093740348C088E9AACF80910D05880F5A
:10304000805FA5CF80910D05813041F0813018F06F
:103050008230C9F506C080910E0399CF80910F038D
:1030600096CF8091100393CF80E891CF84E980932D
:10307000BC008AE090E09093750380937403809184
:103080000D05823060F480910D058F5F80930D05F2
:1030900087E080930A0585EA8093BC0014C01092F3
:1030A0000D0510920A050FC084E98093BC001092B0
:1030B0000A058AE090E09093750380937403109260
:1030C0000B0510920C05FF91EF919F918F910F903E
:1030D0000FBE0F901F9018959FB7F89456985E9A60
:1030E0008AB180638AB98BB18F7C8BB980910001E2
:1030F0008A3011F4539A5B98809180008C70809391
:10310000800080918100837E809381008091810086
:10311000836C80938100809182008F738093820002
:1031200080916F00897F80936F0080916F00816232
:1031300080936F0010920F0510920E059FBF0895A7
:103140001F920F920FB60F9211242F933F935F930C
:103150006F937F938F939F93AF93BF93809110054D
:10316000882391F420910E0530910F0580910E0572
:1031700090910F0568E070E00E949141261B370B8B
:1031800030930F0520930E0510921005BF91AF915B
:103190009F918F917F916F915F913F912F910F90B0
:1031A0000FBE0F901F9018951F920F920FB60F929F
:1031B00011240F931F932F933F934F935F936F931C
:1031C0007F938F939F93AF93BF93CF93DF93EF93AF
:1031D000FF93209186003091870080911105909196
:1031E0001205281B390B80918600909187009093DF
:1031F000120580931105C9018D5494400091130567
:1032000010911405835F9A4188F4043011053CF055
:1032100010927603809110058F5F8093100581E0F6
:1032200090E0909314058093130598C00E3011051B
:103230000CF094C0C9018B5F9040845B914008F012
:1032400072C0E901C25DD140F801EE0FFF1FE159E4
:10325000F84F808191819E01281B390BC90137FFEE
:1032600003C0909581959F4F069784F480910E0539
:1032700090910F05883C91054CF480910E0590913A
:103280000F050A9690930F0580930E05F801EE0F37
:10329000FF1FE159F84F20813181C901880F991F23
:1032A000820F931F8C0F9D1F64E070E00E9491417C
:1032B0009B01CE010196861797071CF421503040E0
:1032C00006C021976C177D0714F42F5F3F4F809144
:1032D0000E0590910F05E801CC0FDD1F833C910591
:1032E000BCF0FE01E159F84F80819181A901481B92
:1032F000590BCA0163E070E00E949141CB01880F35
:10330000991F860F971FC357D84F9983888304C08E
:10331000C357D84F19821882F801EE0FFF1FE159E9
:10332000F84F31832083F8013196F0931405E09330
:103330001305E530F10511F45D9A06C05D98E6309D
:10334000F10511F45C9A01C05C98809100018A300B
:1033500029F4379711F45B9A01C05B9880910E05B0
:1033600090910F05892B49F080910E0590910F05E2
:10337000019790930F0580930E05FF91EF91DF91D8
:10338000CF91BF91AF919F918F917F916F915F91FD
:103390004F913F912F911F910F910F900FBE0F9062
:1033A0001F9018952F923F924F925F926F927F924B
:1033B0008F929F92AF92BF92CF92DF92EF92FF9245
:1033C0000F931F93CF93DF93CDB7DEB762970FB6FE
:1033D000F894DEBF0FBECDBF8091EA049091EB045C
:1033E0000091190510911A05081B190B1093C507B8
:1033F0000093C4078091E8049091E904988B8F872B
:10340000A0911705B0911805BA8BA98BE091E6043D
:10341000F091E704FE87ED878091150590911605E0
:103420009C878B876091F1047091F204882777FD67
:103430008095982F2CE030E040E050E00E9452410F
:103440009B01AC016091AB077091AC07882777FDB9
:103450008095982F620F731F841F951F22E030E024
:1034600040E050E00E94C6413093AC072093AB0788
:103470006091EF047091F004882777FD8095982F74
:103480002CE030E040E050E00E9452419B01AC0152
:103490006091D0077091D107882777FD8095982F8C
:1034A000620F731F841F951F22E030E040E050E060
:1034B0000E94C6413093D1072093D0076091F30456
:1034C0007091F404882777FD8095982F2091BA0792
:1034D0003091BB07442737FD4095542F620F731F6F
:1034E000841F951F22E030E040E050E00E94C6417A
:1034F0003093BB072093BA072091F1043091F20476
:10350000C901880F991F820F931F880F991F880F79
:10351000991FAA2797FDA095BA2F20914F053091AA
:1035200050054091510550915205280F391F4A1FEF
:103530005B1F20934F0530935005409351055093E6
:1035400052052091EF043091F004C901880F991FB2
:10355000820F931F880F991F880F991FAA2797FD25
:10356000A095BA2F209153053091540540915505EF
:1035700050915605280F391F4A1F5B1F2093530592
:103580003093540540935505509356052091F1040E
:103590003091F20480915F0590916005820F931F36
:1035A0009093600580935F052091EF043091F004C3
:1035B0008091610590916205820F931F909362053F
:1035C00080936105809163059091640501969093C5
:1035D0006405809363053801882477FC8094982CD7
:1035E00020904B0530904C0540904D0550904E0575
:1035F000260C371C481C591C20924B0530924C0558
:1036000040924D0550924E058091C7079091C80792
:10361000A091C907B091CA07860D971DA81DB91DB5
:103620008093C7079093C807A093C907B093CA07B0
:10363000803BE3E89E07E8E0AE07E0E0BE0764F009
:10364000805B9348A840B0408093C7079093C80719
:10365000A093C907B093CA078091C7079091C80784
:10366000A091C907B091CA07B7FF0CC080559C470D
:10367000A74FBF4F8093C7079093C807A093C90770
:10368000B093CA07F0919605FA87FF2309F07EC030
:1036900080919705882309F079C08091DF0786FF24
:1036A00075C0E0909E03FF2400E010E020913B05F0
:1036B00030913C0540913D0550913E05C401B30158
:1036C0000E94524120E038E040E050E00E94C641B4
:1036D000CA01B901A80197010E94524120E030E1DE
:1036E00040E050E00E94C64159016A012093D5058F
:1036F0003093D6054093D7055093D80520914305C4
:10370000309144054091450550914605C401B301EF
:103710000E94524120E038E040E050E00E94C64163
:10372000CA01B901A80197010E94524120E030E18D
:1037300040E050E00E94C6412093D1053093D2056D
:103740004093D3055093D405D601C501D7FE07C0D9
:10375000B095A095909581959F4FAF4FBF4F813801
:103760009105A105B10574F457FF07C05095409528
:10377000309521953F4F4F4F5F4F2138310541051F
:103780005105A4F081E080935E0510C01092D10530
:103790001092D2051092D3051092D4051092D5053F
:1037A0001092D6051092D7051092D8058091D505B4
:1037B0009091D605A091D705B091D8058E839F83AF
:1037C000A887B9878091D1059091D205A091D305A2
:1037D000B091D4058A839B83AC83BD8380919F0382
:1037E000682E772488249924C401B3012A813B815F
:1037F0004C815D810E94524120E032E040E050E087
:103800000E94C641EF84F888A989BA89EA1AFB0A9E
:10381000EE81FF81EE0EFF1EE20EF31EF092C30753
:10382000E092C2079701442737FD4095542F8091BD
:10383000470590914805A0914905B0914A05820F2E
:10384000931FA41FB51F8093470590934805A0932D
:103850004905B0934A058091920590919305E81A25
:10386000F90A0027F7FC0095102F809143059091ED
:103870004405A0914505B0914605E80EF91E0A1FC2
:103880001B1FE0924305F0924405009345051093F9
:103890004605A0908103B0908203C0908303D0902E
:1038A0008403AE14BF04C006D106C4F480E197E2DD
:1038B000A0E0B0E08A199B09AC09BD0980934305DB
:1038C00090934405A0934505B09346058093470522
:1038D00090934805A0934905B0934A0522273327C2
:1038E000A9012A193B094C095D0980914305909172
:1038F0004405A0914505B091460582179307A4079A
:10390000B507B4F4D601C50180519742A040B0403C
:103910008093430590934405A0934505B0934605D5
:103920008093470590934805A0934905B0934A05B5
:103930008091E8049091E9040F9734F488E19CEFBA
:103940009093C3078093C2078091E8049091E904A3
:10395000079734F480E398EF9093C3078093C207EE
:10396000F0910001F983FA30A9F48091E804909174
:10397000E904835F934034F088EE93E09093C307AB
:103980008093C2078091E8049091E9048A5F934094
:10399000DCF014C08091E8049091E904855E9740C2
:1039A00034F088EE93E09093C3078093C207809130
:1039B000E8049091E904835F974034F080ED97E04C
:1039C0009093C3078093C207ED84FE848B859C850A
:1039D000E81AF90AAA81BB81EA1AFB0AC401B301F9
:1039E0002E813F81488559850E94524120E032E076
:1039F00040E050E00E94C641E21AF30AF092CE077E
:103A0000E092CD079701442737FD4095542F8091D0
:103A10003F0590914005A0914105B0914205820F6C
:103A2000931FA41FB51F80933F0590934005A0935B
:103A30004105B09342058091940590919505E81A4F
:103A4000F90A0027F7FC0095102F80913B05909113
:103A50003C05A0913D05B0913E05E80EF91E0A1FF8
:103A60001B1FE0923B05F0923C0500933D0510932F
:103A70003E05A0907D03B0907E03C0907F03D09060
:103A80008003AE14BF04C006D106C4F488EA91E6F0
:103A9000A0E0B0E08A199B09AC09BD0980933B0501
:103AA00090933C05A0933D05B0933E0580933F0560
:103AB00090934005A0934105B093420522273327F8
:103AC000A9012A193B094C095D0980913B05909198
:103AD0003C05A0913D05B0913E0582179307A407D0
:103AE000B507B4F4D601C501885A9146A040B0404C
:103AF00080933B0590933C05A0933D05B0933E0514
:103B000080933F0590934005A0934105B0934205F3
:103B10008091E6049091E7040F9734F488E19CEFDC
:103B20009093CE078093CD078091E6049091E704AF
:103B3000079734F480E398EF9093CE078093CD07F6
:103B4000B981BA30A9F48091E6049091E704835FCB
:103B5000934034F088EE93E09093CE078093CD07A6
:103B60008091E6049091E7048A5F9340DCF014C0F2
:103B70008091E6049091E704855E974034F088EEEA
:103B800093E09093CE078093CD078091E6049091C7
:103B9000E704835F974034F080ED97E09093CE0781
:103BA0008093CD0780917A00886C80937A00209270
:103BB0003705309238054092390550923A05809188
:103BC0003B0590913C05A0913D05B0913E05809349
:103BD000270590932805A0932905B0932A05809185
:103BE000430590914405A0914505B0914605809309
:103BF0002F0590933005A0933105B0933205809145
:103C00003F0590914005A0914105B09142058093F8
:103C10002B0590932C05A0932D05B0932E05809134
:103C2000470590914805A0914905B0914A058093B8
:103C3000330590933405A0933505B09336058091F4
:103C4000DF0787FF49C0BA85BB2309F045C08091D3
:103C50009705882309F040C02091CD073091CE0709
:103C6000293C310544F0C901880F991F880F991F1D
:103C7000205233400BC0EFEF28333E076CF4C901EC
:103C8000880F991F880F991F205E3C4F280F391FFE
:103C90003093CE072093CD072091C2073091C30700
:103CA000293C310544F0C901880F991F880F991FDD
:103CB000205233400BC0FFEF28333F076CF4C9019B
:103CC000880F991F880F991F205E3C4F280F391FBE
:103CD0003093C3072093C20762960FB6F894DEBFF5
:103CE0000FBECDBFDF91CF911F910F91FF90EF904D
:103CF000DF90CF90BF90AF909F908F907F906F900C
:103D00005F904F903F902F90089580910E05909175
:103D10000F05813A91050CF439C38091E2078B3F7E
:103D200098F08B3F19F4809168050EC08C3F19F410
:103D300080916A0509C08D3F19F480916C0504C01B
:103D40008E3F21F480916E0580938C038091E10772
:103D50008B3F98F08B3F19F4809168050EC08C3F23
:103D600019F480916A0509C08D3F19F480916C05A2
:103D700004C08E3F21F480916E0580938B03809167
:103D80008B03882319F410928B0305C0843618F036
:103D900084E680938B038091E3078B3F98F08B3F01
:103DA00019F4809168050EC08C3F19F480916A0562
:103DB00009C08D3F19F480916C0504C08E3F21F439
:103DC00080916E0580938D0380918D03882319F473
:103DD00010928D0305C0843618F084E680938D031D
:103DE0008091E5078B3F98F08B3F19F4809168052F
:103DF0000EC08C3F19F480916A0509C08D3F19F4FB
:103E000080916C0504C08E3F21F480916E058093F3
:103E10008E038091EC078B3F98F08B3F19F48091D3
:103E200068050EC08C3F19F480916A0509C08D3F6A
:103E300019F480916C0504C08E3F21F480916E05C9
:103E400080938F038091ED078B3F98F08B3F19F49F
:103E5000809168050EC08C3F19F480916A0509C0F5
:103E60008D3F19F480916C0504C08E3F21F4809140
:103E70006E0580939003809190038B3010F48AE05C
:103E800002C08F3F11F4809390038091EE078B3F27
:103E900098F08B3F19F4809168050EC08C3F19F49F
:103EA00080916A0509C08D3F19F480916C0504C0AA
:103EB0008E3F21F480916E05809391038091F307EA
:103EC0008B3F98F08B3F19F4809168050EC08C3FB2
:103ED00019F480916A0509C08D3F19F480916C0531
:103EE00004C08E3F21F480916E05809393038091EE
:103EF000F4078B3F98F08B3F19F4809168050EC052
:103F00008C3F19F480916A0509C08D3F19F48091A6
:103F10006C0504C08E3F21F480916E05809394035C
:103F20008091F5078B3F98F08B3F19F480916805DD
:103F30000EC08C3F19F480916A0509C08D3F19F4B9
:103F400080916C0504C08E3F21F480916E058093B2
:103F500095038091F6078B3F98F08B3F19F4809181
:103F600068050EC08C3F19F480916A0509C08D3F29
:103F700019F480916C0504C08E3F21F480916E0588
:103F8000809396038091F7078B3F98F08B3F19F44D
:103F9000809168050EC08C3F19F480916A0509C0B4
:103FA0008D3F19F480916C0504C08E3F21F48091FF
:103FB0006E0580939703809107088B3F98F08B3FA5
:103FC00019F4809168050EC08C3F19F480916A0540
:103FD00009C08D3F19F480916C0504C08E3F21F417
:103FE00080916E0580939803809108088B3F98F02C
:103FF0008B3F19F4809168050EC08C3F19F48091B5
:104000006A0509C08D3F19F480916C0504C08E3F8C
:1040100021F480916E0580939903809109088B3F6C
:1040200098F08B3F19F4809168050EC08C3F19F40D
:1040300080916A0509C08D3F19F480916C0504C018
:104040008E3F21F480916E0580939A0380910A0837
:104050008B3F98F08B3F19F4809168050EC08C3F20
:1040600019F480916A0509C08D3F19F480916C059F
:1040700004C08E3F21F480916E0580939B03809154
:10408000F8078B3F98F08B3F19F4809168050EC0BC
:104090008C3F19F480916A0509C08D3F19F4809115
:1040A0006C0504C08E3F21F480916E0580939C03C3
:1040B0008091FD078B3F98F08B3F19F48091680544
:1040C0000EC08C3F19F480916A0509C08D3F19F428
:1040D00080916C0504C08E3F21F480916E05809321
:1040E0009D03809100088B3F98F08B3F19F48091DD
:1040F00068050EC08C3F19F480916A0509C08D3F98
:1041000019F480916C0504C08E3F21F480916E05F6
:1041100080939E03809101088B3F98F08B3F19F4A8
:10412000809168050EC08C3F19F480916A0509C022
:104130008D3F19F480916C0504C08E3F21F480916D
:104140006E0580939F03809106088B3F98F08B3F0C
:1041500019F4809168050EC08C3F19F480916A05AE
:1041600009C08D3F19F480916C0504C08E3F21F485
:1041700080916E058093A00380910C088B3F98F08E
:104180008B3F19F4809168050EC08C3F19F4809123
:104190006A0509C08D3F19F480916C0504C08E3FFB
:1041A00021F480916E058093A2038091A203823056
:1041B00010F481E002C08F3F11F48093A20380913C
:1041C0000E088B3F98F08B3F19F4809168050EC064
:1041D0008C3F19F480916A0509C08D3F19F48091D4
:1041E0006C0504C08E3F21F480916E058093A3037B
:1041F0008091A303823010F481E002C08F3F11F45C
:104200008093A30380910F088B3F98F08B3F19F4A4
:10421000809168050EC08C3F19F480916A0509C031
:104220008D3F19F480916C0504C08E3F21F480917C
:104230006E058093A403809110088B3F98F08B3F0C
:1042400019F4809168050EC08C3F19F480916A05BD
:1042500009C08D3F19F480916C0504C08E3F21F494
:1042600080916E058093A503809111088B3F98F093
:104270008B3F19F4809168050EC08C3F19F4809132
:104280006A0509C08D3F19F480916C0504C08E3F0A
:1042900021F480916E058093A603809112088B3FD4
:1042A00098F08B3F19F4809168050EC08C3F19F48B
:1042B00080916A0509C08D3F19F480916C0504C096
:1042C0008E3F21F480916E058093A703809113089F
:1042D0008B3F98F08B3F19F4809168050EC08C3F9E
:1042E00019F480916A0509C08D3F19F480916C051D
:1042F00004C08E3F21F480916E058093A8038091C5
:1043000014088B3F98F08B3F19F4809168050EC01C
:104310008C3F19F480916A0509C08D3F19F4809192
:104320006C0504C08E3F21F480916E058093A90333
:10433000809117088B3F98F08B3F19F480916805A6
:104340000EC08C3F19F480916A0509C08D3F19F4A5
:1043500080916C0504C08E3F21F480916E0580939E
:10436000A1036091930370E080E090E00E948A3D99
:1043700027E137EB41ED58E30E94EF40609387035C
:10438000709388038093890390938A0308958091A2
:10439000670580FD31C01092CF071092C6071092BA
:1043A000B1071092BC071092BD071092D6078091FA
:1043B000CC04882331F08093BC078091BC078093A4
:1043C000C6078091CD04882331F08093B107809196
:1043D000B1078093CF078091CE04882311F080939A
:1043E000D6078091CF04882311F08093BD07809178
:1043F0006705857F8093670510920A050E9428173C
:104400000895809100018D3010F00E94401080913D
:104410007A00877380937A008091E6049091E70494
:104420009093CE078093CD078091E8049091E904A2
:104430009093C3078093C2078091EA049091EB04A4
:104440009093C5078093C4076091F1047091F204C2
:10445000882777FD8095982F2CE030E040E050E0F1
:104460000E9452417093AC076093AB076091EF04D8
:104470007091F004882777FD8095982F0E94524113
:104480007093D1076093D0078091F3049091F40466
:104490009093BB078093BA0780917A00886C8093D1
:1044A0007A006091020870E080E090E024EC39E04E
:1044B00040E050E00E94524160937D0370937E0380
:1044C00080937F03909380036091030870E080E005
:1044D00090E00E9452416093810370938203809325
:1044E00083039093840308951092200510921F0572
:1044F000109222051092210580E090E0A0E0B0E04B
:104500008093230590932405A0932505B093260559
:1045100010921605109215051092180510921705A5
:1045200010921A051092190510929E0310929F0383
:104530000E94012284E690E00E94CF0B0E9401229B
:104540008091DF0780FF10C08091150390911603C2
:10455000875B934038F480911503909116038E5E2B
:10456000924010F40E94FB104091E6045091E70441
:1045700050931605409315052091E8043091E90405
:1045800030931805209317058091EA049091EB046D
:1045900090931A058093190530931C0520931B05F1
:1045A00050931E0540931D0584E00E94123A8050EE
:1045B000944058F18091D0079091D10797FF03C0A4
:1045C000909581959F4F6CE070E00E9491417093AF
:1045D0002205609321058091AB079091AC0797FF6E
:1045E00003C0909581959F4F6CE070E00E949141CF
:1045F0007093200560931F056091E4047091E504B9
:10460000882777FD8095982F17C084E00E94123A82
:104610009093200580931F0586E00E94123A9093A4
:1046200022058093210588E00E94123AAA2797FD6F
:10463000A095BA2FBC01CD010E943740609323059D
:1046400070932405809325059093260510923B05D1
:1046500010923C0510923D0510923E0510923F05C8
:1046600010924005109241051092420510924305A8
:104670001092440510924505109246051092470588
:10468000109248051092490510924A0510924B0568
:1046900010924C0510924D0510924E051092CE07C7
:1046A0001092CD071092C3071092C2071092C5074F
:1046B0001092C40784E690E00E94CF0B8091110312
:1046C00090911203A0911303B0911403909361078A
:1046D000809360071092F7041092F6041092570529
:1046E000109258051092590510925A05809177033F
:1046F0009091780390937A038093790382E390E01A
:104700009093E0048093DF046091020870E080E001
:1047100090E024EC39E040E050E00E9452416856BD
:10472000754C8F4F9F4F60937D0370937E038093F2
:104730007F03909380036091030870E080E090E035
:104740000E9452416856754C8F4F9F4F6093810372
:104750007093820380938303909384031092860363
:1047600010928503109281051092800510928305A6
:10477000109282056091770370917803882777FD06
:104780008095982F2EE036E040E050E00E945241A4
:104790006093C7077093C8078093C9079093CA07AF
:1047A0001092CC071092CB078091670584608093AC
:1047B000670508951F93182F0EC08091670580FD2F
:1047C0000CC084E690E09093E0048093DF048AEFCD
:1047D00090E00E94ED0B115080F71F910895809199
:1047E000D707E82FF0E0EE0FFF1FE159F84F808167
:1047F00091818D5E9F4F14F01092AA038081918168
:104800008A5B9F4FDCF48091AA038823B9F481E08E
:104810008093AA0380915D058F5F80935D058091F1
:104820005D05853028F480915D050E94DA230895A6
:1048300088EE93E09093E0048093DF0408952F9234
:104840003F924F925F926F927F928F929F92AF9220
:10485000BF92CF92DF92EF92FF920F931F93CF936D
:10486000DF93CDB7DEB7E4970FB6F894DEBF0FBE87
:10487000CDBF0E94D219409100014C3010F4299A0A
:1048800001C0299820917E0530917F058091E9072C
:10489000682F70E0665F7F4F7C8B6B8B62177307AE
:1048A00014F43C8B2B8B80910E0590910F0588376B
:1048B00091050CF072C080910301882399F48091D6
:1048C0000403909105038F5F9F4F61F488E99AE399
:1048D0009093E0048093DF0480E09CE090930503D4
:1048E000809304038091BB059091BC05009731F043
:1048F00001979093BC058093BB0505C08091670527
:104900008E7E809367054A3011F4289A01C028985A
:104910008091650590916605895E934008F429C4ED
:104920008091F007E82FF0E0FC8BEB8B809167051E
:10493000806180936705E091D7072E2F30E0220F2A
:10494000331FF901E357F84F11821082A091D80765
:10495000B0E0AA0FBB1FFD01E357F84F1182108290
:10496000E091DA074E2F50E0440F551FCA018357DC
:10497000984FFC01118210822159384FF9011182A0
:104980001082A159B84F11961C921E924159584F4E
:10499000DA0111961C921E92F4C380910E0590913B
:1049A0000F058D3891050CF4ECC3809167058F7E5F
:1049B000809367058091F10722E3829FC001112453
:1049C0009093BC058093BB05EB89FC89B9978CF06B
:1049D0008091670580FF0DC0809165059091660507
:1049E000FFEF8F3F9F0729F0019690936605809314
:1049F000650580916505909166058F3F910509F0E9
:104A000070F51092CD051092CE051092CF05109240
:104A1000D0051092C9051092CA051092CB051092CC
:104A2000CC0510927D0510927C058A3F9105E1F43A
:104A300081E090E09093B3058093B20510924B050E
:104A400010924C0510924D0510924E051092C5051E
:104A50001092C6051092C7051092C80505C0809136
:104A6000670582608093670520916805309169052C
:104A70008091DB07E82FF0E0EE0FFF1FE159F84FC0
:104A80008081918182599F4F281739071CF42F5F2D
:104A90003F4F0CC08081918182599F4F82179307AD
:104AA0004CF42115310531F0215030403093690527
:104AB0002093680520916A0530916B058091DC0791
:104AC000E82FF0E0EE0FFF1FE159F84F8081918150
:104AD00082599F4F281739071CF42F5F3F4F0CC096
:104AE0008081918182599F4F821793074CF4211541
:104AF000310531F02150304030936B0520936A0529
:104B000020916C0530916D058091DD07E82FF0E074
:104B1000EE0FFF1FE159F84F8081918182599F4F1D
:104B2000281739071CF42F5F3F4F0CC080819181FB
:104B300082599F4F821793074CF42115310531F0AC
:104B40002150304030936D0520936C0520916E0507
:104B500030916F058091DE07E82FF0E0EE0FFF1F28
:104B6000E159F84F8081918182599F4F2817390769
:104B70001CF42F5F3F4F0CC08081918182599F4F61
:104B8000821793074CF42115310531F02150304044
:104B900030936F0520936E0520917005309171055B
:104BA000809181079091820782599F4F281739077A
:104BB0001CF42F5F3F4F0EC08091810790918207B8
:104BC00082599F4F821793074CF42115310531F01C
:104BD000215030403093710520937005209172056B
:104BE00030917305809183079091840782599F4F7C
:104BF000281739071CF42F5F3F4F0EC080918307A1
:104C00009091840782599F4F821793074CF4211586
:104C1000310531F0215030403093730520937205F7
:104C200020917405309175058091850790918607D4
:104C300082599F4F281739071CF42F5F3F4F0EC032
:104C4000809185079091860782599F4F821793071D
:104C50004CF42115310531F0215030403093750569
:104C60002093740520917605309177058091870710
:104C70009091880782599F4F281739071CF42F5F9E
:104C80003F4F0EC0809187079091880782599F4FB0
:104C9000821793074CF42115310531F02150304033
:104CA000309377052093760580916805909169058A
:104CB00097FF05C010926905109268050AC08F3FE2
:104CC000910539F034F08FEF90E09093690580936F
:104CD000680580916A0590916B0597FF05C0109259
:104CE0006B0510926A050AC08F3F910539F034F0C8
:104CF0008FEF90E090936B0580936A0580916C052F
:104D000090916D0597FF05C010926D0510926C058E
:104D10000AC08F3F910539F034F08FEF90E0909307
:104D20006D0580936C0580916E0590916F0597FFDE
:104D300005C010926F0510926E050AC08F3F910555
:104D400039F034F08FEF90E090936F0580936E050B
:104D5000809170059091710597FF05C010927105C3
:104D6000109270050AC08F3F910539F034F08FEF33
:104D700090E09093710580937005809172059091F9
:104D8000730597FF05C010927305109272050AC053
:104D90008F3F910539F034F08FEF90E090937305D9
:104DA00080937205809174059091750597FF05C0F9
:104DB00010927505109274050AC08F3F910539F065
:104DC00034F08FEF90E09093750580937405809197
:104DD00076059091770597FF05C0109277051092A0
:104DE00076050AC08F3F910539F034F08FEF90E0DF
:104DF0009093770580937605E091D907F0E0EE0F68
:104E0000FF1FE159F84F80819181813591050CF4A4
:104E100015C18091670580FD11C18091DA07E82FE7
:104E2000F0E0EE0FFF1FE159F84F808191818C3443
:104E300091050CF4C3C08091BA058F5F8093BA05C9
:104E4000893C08F4FBC01092BA054C3010F4299844
:104E500001C0299A10926605109265058091D707C6
:104E6000282F30E0D901AA0FBB1FA159B84F8D914F
:104E70009C911197873491059CF48091D807E82F75
:104E8000F0E0EE0FFF1FE159F84F8081918197FF0D
:104E900003C0909581959F4F873491050CF46BC0AA
:104EA0008091D807682F70E0DB01AA0FBB1FA159C2
:104EB000B84F8D919C911197873491053CF0F90181
:104EC000EE0FFF1FE159F84F808191818D919C91E8
:104ED0008734910564F0F901EE0FFF1FE159F84F97
:104EE000808191818734910514F042E001C041E056
:104EF000FB01EE0FFF1FE159F84F8081918186344D
:104F000091055CF4F901EE0FFF1FE159F84F808124
:104F10009181873491050CF043E0FB01EE0FFF1FF8
:104F2000E159F84F808191818A5B9F4F5CF4F901D0
:104F3000EE0FFF1FE159F84F808191818734910571
:104F40000CF044E0660F771F6159784FDB018D91BB
:104F50009C918A5B9F4F5CF4220F331F2159384F7D
:104F6000F90180819181863491050CF445E0842F0C
:104F70000E94223A1CC08091DF078872C1F08081B4
:104F8000918197FF03C0909581959F4F44977CF442
:104F90008D919C918A5B9F4F54F481E080935D05D5
:104FA00088EE93E09093E0048093DF0447C00E9472
:104FB000593C0E94423A0E94742239C080819181FA
:104FC000855B9F4FCCF58091BA058F5F8093BA05C2
:104FD000893CA0F11092BA054C3010F4299801C018
:104FE000299A6FEF7FEF84E00E941A3A10926605CB
:104FF000109265050E94742260911F057091200532
:1050000084E00E941A3A609121057091220586E0A1
:105010000E941A3A6091230570912405809125051C
:10502000909126050E94094088E00E941A3A0E9449
:10503000593C0E94DA2302C01092BA05E091D907C8
:10504000F0E0EE0FFF1FE159F84F808191818B5AFC
:105050009F4F0CF096C08091DA07482F50E0FA017C
:10506000EE0FFF1FE159F84F80819181855B9F4FC3
:105070000CF066C08091B9058F5F8093B905893CBB
:1050800008F460C01092B90581E090E09093660545
:10509000809365058091670589608093670510920C
:1050A000C5051092C6051092C7051092C80510924A
:1050B0004B0510924C0510924D0510924E05109222
:1050C0003B0510923C0510923D0510923E05109252
:1050D00043051092440510924505109246058091B3
:1050E000270590912805A0912905B0912A05809364
:1050F0003F0590934005A0934105B09342058091F0
:105100002F0590913005A0913105B0913205809323
:10511000470590934805A0934905B0934A0510921E
:10512000CD051092CE051092CF051092D0051092A9
:10513000C9051092CA051092CB051092CC0502C089
:105140001092B905440F551F4159584FDA018D91FE
:105150009C918C3491059CF08091B8058F5F809371
:10516000B805893C70F01092B8051092660510924F
:105170006505809167058E7F8093670502C0109258
:10518000B8058091760381508093760380917603F1
:105190008F3F21F08091670584FF8FC30E94851E99
:1051A000E0917805F0917905FCABEBAB8091D707E6
:1051B000E82EFF24D701AA0FBB1FCD018159984FBC
:1051C000FC01808191819AAB89AB8091E607882EA2
:1051D0009924A357B84F0D90BC91A02DB8ABAFA7A1
:1051E0008091E707282F30E03EA72DA7409180054A
:1051F000509181055CA74BA760917A0570917B0562
:105200007AA769A78091D807082F10E0C801880FF6
:10521000991FDC01A159B84F0D90BC91A02DB8A7E2
:10522000AFA38357984FDC018D919C919EA38DA3D2
:10523000E0918205F0918305FCA3EBA3E091DA07EE
:10524000AE2FB0E0AA0FBB1FA159B84F0D90BC9173
:10525000A02DBAA3A9A3E091D907F0E0EE0FFF1F9C
:10526000E159F84FC080D18028E730E0C20ED31E4C
:10527000D0927F05C0927E056091900370E080E03F
:1052800090E00E948A3D20E030E040E251E40E943C
:10529000383F20E030E040E85CE30E94EF401B0133
:1052A0002C016093D2077093D3078093D407909317
:1052B000D5076091910370E080E090E00E948A3D04
:1052C00020E030EE4BE256E40E949C3F6093BE0724
:1052D0007093BF078093C0079093C1072091D104BA
:1052E000222331F08AE090E09093E0048093DF0481
:1052F000E22F22FF09C08091A103482F50E0440F04
:10530000551F440F551F10C023FD03C040E050E05F
:105310000BC08091A10390E0880F991F880F991FFF
:1053200044275527481B590B209188053091890542
:10533000C901B3E0880F991FBA95E1F7821B930B5F
:10534000840F951F68E070E00E9491413B017093CB
:10535000890560938805E4FF09C08091A103482F67
:1053600050E0440F551F440F551F10C0E5FD03C00A
:1053700040E050E00BC08091A10390E0880F991F9E
:10538000880F991F44275527481B590B80918A0580
:1053900090918B059C01E3E0220F331FEA95E1F722
:1053A000281B390BCA01820F931F68E070E00E942E
:1053B00091415B0170938B0560938A058091D004C5
:1053C000282F83FF03C082E390E004C082FF07C060
:1053D0008EEC9FEF90938D0580938C0504C0109206
:1053E0008D0510928C0521FF09C080918503909155
:1053F00086030196909386038093850324FF09C05A
:105400008091850390918603019790938603809302
:10541000850349A95AA9489DC001499D900D589DF1
:10542000900D11242BA93CA9220F331F6BA97CA935
:10543000260F371FEFA5F8A94DA55EA5E49FD00163
:10544000E59FB00DF49FB00D11246BA57CA5A61BA4
:10545000B70BBCABABAB820F931F64E070E00E9454
:1054600091418BA99CA9860F971F9CAB8BABC30165
:1054700062E070E00E949141ABA9BCA9A60FB71FE2
:10548000BCABABABB0937905A0937805EFA1F8A5C1
:10549000E89DC001E99D900DF89D900D112429A56E
:1054A0003AA5220F331F49A55AA5240F351F6DA118
:1054B0007EA1ADA5BEA56A9F30016B9F700C7A9F3F
:1054C000700C1124EBA1FCA16E1A7F0A820F931FAE
:1054D00064E070E00E949141660E771EC50162E0B3
:1054E00070E00E949141660E771E70927B0560927B
:1054F0007A0520918C0530918D05220F331F220FE4
:10550000331F49A15AA1241B350B30937D052093ED
:105510007C058091850680FF56C08091A10381386B
:1055200008F451C080917E06992787FD9095BC01B3
:10553000689DC001699D900D789D900D1124ABA9C7
:10554000BCA9A80FB91FB0937905A09378058091E5
:105550007F06992787FD9095FC01E89DC001E99D94
:10556000900DF89D900D1124680E791E70927B05A8
:1055700060927A0580918006992787FD9095280F83
:10558000391F30937D0520937C052091E40730E09E
:1055900080918206992787FD9095AC01249FC001D8
:1055A000259F900D349F900D112490938603809336
:1055B00085038091810690E08C159D0524F49093DD
:1055C0007F0580937E0580917E0590917F0597FFF2
:1055D00004C010927F0510927E058091DF0782FF44
:1055E0000CC080E090E0A0E0B0E08093BE07909314
:1055F000BF07A093C007B093C10720E030E040E0B0
:1056000050E0C201B1010E947240882364F480E03E
:1056100090E0A0E0B0E08093D2079093D307A093EE
:10562000D407B093D50720E030E040E050E060912F
:10563000BE077091BF078091C0079091C1070E947B
:105640007240882364F480E090E0A0E0B0E08093B2
:10565000BE079093BF07A093C007B093C107E09126
:105660007805F09179052091840530918505CF0169
:1056700064E070E00E94914177FF03C070956195EE
:105680007F4F26173707C4F4CF01F7FF03C090956B
:1056900081959F4F64E070E00E9491417093850571
:1056A00060938405653671056CF084E690E0909314
:1056B00085058093840506C02150304030938505D0
:1056C00020938405E0917A05F0917B052091860571
:1056D00030918705CF0164E070E00E94914177FF2F
:1056E00003C0709561957F4F26173707C4F4CF012B
:1056F000F7FF03C0909581959F4F64E070E00E9492
:1057000091417093870560938605653671056CF04D
:1057100084E690E0909387058093860506C021502B
:1057200030403093870520938605F801EE0FFF1F68
:10573000E159F84F208131818091FE07482F50E0D8
:105740004217530744F48091180882FF04C081E097
:105750008093980515C080919805882389F0F801F9
:10576000EE0FFF1FE159F84F208131818091FF0733
:10577000BA01681B71092617370714F410929805AF
:10578000F801EE0FFF1FE159F84F808191816627E4
:105790007727641B750B8617970744F480911808C8
:1057A00083FF04C081E08093990515C0809199051D
:1057B000882389F0000F111F0159184FD8012D912E
:1057C0003C918091FF0790E0841B950B8217930713
:1057D00014F410929905F701EE0FFF1FE159F84FED
:1057E000808191814817590744F48091180880FFFF
:1057F00004C081E080939B0515C080919B058823A0
:1058000089F0F701EE0FFF1FE159F84F2081318138
:105810008091FF07FA01E81BF1092E173F0714F4E6
:1058200010929B05F701EE0FFF1FE159F84F8081A1
:1058300091818617970744F48091180881FF04C06E
:1058400081E080939A0517C080919A05882399F08A
:10585000EE0CFF1C2FE637E0E20EF31ED7012D9170
:105860003C918091FF0790E0841B950B8217930772
:1058700014F410929A0580919805882321F4809160
:105880009905882321F081E08093970502C010924A
:10589000970580919B05882321F480919A058823A0
:1058A00051F081E08093960510929705109298052B
:1058B0001092990502C01092960580919705882351
:1058C00021F480919605882351F08091FD0790E0A6
:1058D000EB89FC898E179F0714F49C8B8B8B80912E
:1058E000670584FF30C010927D0510927C051092F0
:1058F00079051092780510927B0510927A0580E068
:1059000090E0A8ECBFE38093D2079093D307A093D5
:10591000D407B093D5078BE09CEBA2E3BCE3809364
:10592000BE079093BF07A093C007B093C107109222
:105930009705109296051092850510928405109295
:105940008705109286052091270530912805409102
:10595000290550912A052D833E834F8358878091D6
:10596000AD079091AE07A091AF07B091B007820F3D
:10597000931FA41FB51F8093AD079093AE07A0930C
:10598000AF07B093B00740912F055091300560915B
:105990003105709132054F87588B698B7A8B8091D6
:1059A000B4079091B507A091B607B091B707840FDF
:1059B000951FA61FB71F8093B4079093B507A093B8
:1059C000B607B093B70790909605992029F4809177
:1059D0009705882309F44FC01092F9041092F80437
:1059E00010924F05109250051092510510925205D9
:1059F00010925305109254051092550510925605B9
:105A00001092AD071092AE071092AF071092B00738
:105A10001092B4071092B5071092B6071092B7070C
:105A200080913B0590913C05A0913D05B0913E05CC
:105A300080933F0590934005A0934105B0934205A4
:105A40008091430590914405A0914505B09146058C
:105A50008093470590934805A0934905B0934A0564
:105A6000109295051092940510929305109292054C
:105A7000992009F0EFC080919705882309F0EAC0CA
:105A8000E090EB07FF2400E010E06D817E818F81C4
:105A90009885A80197010E94C6418091AB0790911B
:105AA000AC07AA2797FDA095BA2F281B390B4A0BE4
:105AB0005B0BCA01B90120E130E040E050E00E94F8
:105AC000C64159016A016F85788989899A89A80137
:105AD00097010E94C6418091D0079091D107AA27D3
:105AE00097FDA095BA2F281B390B4A0B5B0BCA01F7
:105AF000B90120E130E040E050E00E94C641790168
:105B00008A018091840590918505813491053CF44A
:105B1000809186059091870581349105A4F0C60196
:105B2000B50123E030E040E050E00E94C641590159
:105B30006A01C801B70123E030E040E050E00E9474
:105B4000C64179018A01E091DA07F0E0EE0FFF1F0C
:105B5000E159F84F0190F081E02DF7FF03C0F09577
:105B6000E195FF4F7A97A4F0C601B50123E030E03C
:105B700040E050E00E94C64159016A01C801B701E6
:105B800023E030E040E050E00E94C64179018A0104
:105B900051E2A516B104C104D10434F0E0E2AE2E06
:105BA000B12CC12CD12C11C060EEA6166FEFB60639
:105BB0006FEFC6066FEFD60644F470EEA72E7FEFA8
:105BC000B72E7FEFC72E7FEFD72E71E2E716F104D5
:105BD0000105110534F060E2E62EF12C012D112DA6
:105BE00011C080EEE8168FEFF8068FEF08078FEFF1
:105BF000180744F450EEE52E5FEFF52E5FEF052F0A
:105C00005FEF152F80913B0590913C05A0913D05DC
:105C1000B0913E058A199B09AC09BD0980933B05EB
:105C200090933C05A0933D05B0933E0580914305BC
:105C300090914405A0914505B09146058E199F09A4
:105C4000A00BB10B8093430590934405A0934505A9
:105C5000B09346058091F8049091F9048F3F910527
:105C600009F008F419C4992009F0B0C38091970590
:105C7000882309F0ABC380915E05882309F0A6C391
:105C80006091AD077091AE078091AF079091B0071A
:105C900020E031E040E050E00E94C64119012A01B5
:105CA0002093AD073093AE074093AF075093B007F2
:105CB0006091B4077091B5078091B6079091B707CE
:105CC00020E031E040E050E00E94C6412D8F3E8F41
:105CD0004F8F58A32093B4073093B5074093B6076E
:105CE0005093B707E090EB07FF2400E010E020910D
:105CF0004F05309150054091510550915205C80112
:105D0000B7010E94524120E031E040E050E00E94A3
:105D1000C64159016A0120934F05309350054093C5
:105D200051055093520520915305309154054091EF
:105D3000550550915605C801B7010E94524120E017
:105D400031E040E050E00E94C64139014A01209311
:105D50005305309354054093550550935605E090F4
:105D60000408FF2400E010E0C201B1016A197B09B8
:105D70008C099D09A80197010E94C641CA01B90179
:105D800020E031E040E050E00E94C64169013093DC
:105D90009505209394056D8D7E8D8F8D98A1661944
:105DA000770988099909A80197010E94C641CA018B
:105DB000B90120E031E040E050E00E94C641890195
:105DC00030939305209392058091840590918505E9
:105DD00081349105C4F480918605909187058134C2
:105DE00091058CF4E091DA07F0E0EE0FFF1FE15926
:105DF000F84F0190F081E02DF7FF03C0F095E19599
:105E0000FF4F7A9794F0C60162E070E00E949141E2
:105E10007093950560939405C80162E070E00E945C
:105E200091417093930560939205E0902B05F0905B
:105E30002C0500912D0510912E052D813E814F815D
:105E40005885E21AF30A040B150BE092C105F09293
:105E5000C2050093C3051093C40580913F0590913E
:105E60004005A0914105B09142058E199F09A00BF4
:105E7000B10B80933F0590934005A0934105B093EB
:105E80004205A0903305B0903405C0903505D09000
:105E900036054F85588969897A89A41AB50AC60AD0
:105EA000D70AA092BD05B092BE05C092BF05D092A0
:105EB000C0058091470590914805A0914905B09192
:105EC0004A058A199B09AC09BD098093470590933F
:105ED0004805A0934905B0934A052091CB0730911E
:105EE000CC07213831054CF08091190590911A05A5
:105EF000019690931A058093190520583F4F4CF452
:105F00008091190590911A05019790931A05809335
:105F100019051092CC071092CB0781E090E0909386
:105F2000A9058093A8051092AE051092AF051092B6
:105F3000B0051092B1058091A0059091A105A091A6
:105F4000A205B091A30582199309A409B509815E40
:105F5000914BAF4FBF4F8F539C49A040B04008F0CA
:105F6000C1C071E0E71670E1F70670E0070770E066
:105F700017070CF452C08091A705882309F449C083
:105F8000D801C7013CE0B595A795979587953A95B7
:105F9000D1F701969093A9058093A805D801C70170
:105FA00023E0B595A795979587952A95D1F7809386
:105FB000AE059093AF05A093B005B093B105895895
:105FC0009341A040B04064F088E893E1A0E0B0E0E5
:105FD0008093AE059093AF05A093B005B093B10543
:105FE0006091AE057091AF058091B0059091B105BB
:105FF00020E031E040E050E00E94C64180919405ED
:1060000090919505820F931F909395058093940529
:1060100066C081E08093A70562C01092A705F0E0FA
:10602000EF16F0EFFF06FFEF0F07FFEF1F070CF073
:1060300056C08091A605882309F44DC0882799276A
:10604000DC018E199F09A00BB10BFCE0B595A7955B
:1060500097958795FA95D1F701969093A905809326
:10606000A805C801B70128E030E040E050E00E94F8
:10607000C6412093AE053093AF054093B0055093D1
:10608000B10528573C4E4F4F5F4F64F488E79CEEB4
:10609000AFEFBFEF8093AE059093AF05A093B0052F
:1060A000B093B1056091AE057091AF058091B005D8
:1060B0009091B10520E031E040E050E00E94C641FF
:1060C0008091940590919505820F931F909395056B
:1060D0008093940511C081E08093A6050DC01092B5
:1060E000A6050AC01092A9051092A80588EE93E0B3
:1060F00090937C0380937B0380910508882E9924DC
:106100008091A8059091A9058816990624F490928B
:10611000A9058092A80571E0E71674E0F70670E023
:10612000070770E0170774F0809115059091160528
:106130002091A8053091A905820F931F9093160511
:106140008093150580E0E8168CEFF8068FEF0807BE
:106150008FEF180774F48091150590911605209122
:10616000A8053091A905821B930B90931605809387
:10617000150581E090E09093A9058093A805109201
:10618000AA051092AB051092AC051092AD05809156
:106190009C0590919D05A0919E05B0919F052D8D28
:1061A0003E8D4F8D58A1821B930BA40BB50B815EC6
:1061B000914BAF4FBF4F8F539C49A040B04008F068
:1061C000C1C041E0A41640E1B40640E0C40640E08E
:1061D000D4060CF452C08091A505882309F449C067
:1061E000D601C501ECE0B595A79597958795EA95F9
:1061F000D1F701969093A9058093A805D601C50112
:1062000073E0B595A795979587957A95D1F7809383
:10621000AA059093AB05A093AC05B093AD05895842
:106220009341A040B04064F088E893E1A0E0B0E082
:106230008093AA059093AB05A093AC05B093AD05F0
:106240006091AA057091AB058091AC059091AD0568
:1062500020E031E040E050E00E94C641809192058C
:1062600090919305820F931F9093930580939205CD
:1062700066C081E08093A50562C01092A50560E02C
:10628000A61660EFB6066FEFC6066FEFD6060CF0E7
:1062900056C08091A405882309F44DC0882799270A
:1062A000DC018A199B09AC09BD096CE0B595A7957D
:1062B000979587956A95D1F701969093A905809354
:1062C000A805C601B50128E030E040E050E00E949A
:1062D000C6412093AA053093AB054093AC0550937B
:1062E000AD0528573C4E4F4F5F4F64F488E79CEE56
:1062F000AFEFBFEF8093AA059093AB05A093AC05D9
:10630000B093AD056091AA057091AB058091AC0585
:106310009091AD0520E031E040E050E00E94C641A0
:106320008091920590919305820F931F909393050E
:106330008093920511C081E08093A4050DC0109256
:10634000A4050AC01092A9051092A80588EE93E052
:1063500090937C0380937B038091A8059091A9057D
:106360008816990624F49092A9058092A80581E0E8
:10637000A81684E0B80680E0C80680E0D80674F06D
:1063800080911705909118052091A8053091A905D5
:10639000820F931F909318058093170590E0A9161C
:1063A0009CEFB9069FEFC9069FEFD906CCF4809108
:1063B0001705909118052091A8053091A905821B19
:1063C000930B90931805809317050AC010929305BC
:1063D00010929205109295051092940510925E0508
:1063E00020E030E040E050E06091BE077091BF07D0
:1063F0008091C0079091C1070E947240882341F4A8
:1064000010929305109292051092950510929405A2
:106410008091AD079091AE07A091AF07B091B00702
:106420008093A0059093A105A093A205B093A30526
:106430008091B4079091B507A091B607B091B707C6
:1064400080939C0590939D05A0939E05B0939F0516
:1064500010924F051092500510925105109252055E
:10646000109253051092540510925505109256053E
:106470001092AD071092AE071092AF071092B007BE
:106480001092B4071092B5071092B6071092B70792
:106490001092F9041092F804C0907C05D0907D050C
:1064A0008601D7FE04C0002711270C191D090031F1
:1064B000110584F088EE93E090937C0380937B0336
:1064C0008091DF0784FD06C081E090E09093B305E2
:1064D0008093B205E090E807B601882777FD8095A4
:1064E000982F2E2D30E040E050E00E94524198015C
:1064F000442737FD4095542F0E94524120E032E05E
:1065000040E050E00E94C64189019A01FF24EC9CC2
:10651000C001ED9C900DFC9C900D112464E070E096
:106520000E949141600F711F882777FD8095982FF9
:106530006093C5057093C6058093C7059093C80501
:1065400020914B0530914C0540914D0550914E05E1
:10655000261B370B480B590B20934B0530934C05EA
:1065600040934D0550934E052155334C40405040CB
:1065700064F080E593ECA0E0B0E080934B0590934D
:106580004C05A0934D05B0934E0580914B0590911D
:106590004C05A0914D05B0914E05805B9C43AF4FDB
:1065A000BF4F64F480EB9CE3AFEFBFEF80934B05EC
:1065B00090934C05A0934D05B0934E058091DF0755
:1065C000887209F458C180915D05882339F0809163
:1065D000670580FD03C00E94EF234DC16D817E8160
:1065E0008F81988520E032E040E050E00E94C64173
:1065F000890137FF03C0109501951F4F6F8578897A
:1066000089899A8920E032E040E050E00E94C6414A
:10661000690137FF04C0D094C194D108D394C01647
:10662000D1060CF46801809177039091780397FF6D
:1066300003C0AA24BB242CC0E0907703F090780319
:106640002CE132E0E20EF31E0027F7FC0095102F3C
:106650006091C7077091C8078091C9079091CA07D8
:106660002EE036E040E050E00E94C641E21AF30A14
:10667000040B150BC801B70128E631E040E050E0FB
:106680000E94C6415CE4A52E5FEFB52EA60EB71E94
:10669000E0907B03F0907C03E114F10481F539E193
:1066A000C316D10464F58091CB079091CC078A0D75
:1066B0009B1D9093CC078093CB078091B20590915E
:1066C000B305892BE1F088EC90E09093E00480938F
:1066D000DF046091C7077091C8078091C907909146
:1066E000CA072EE036E040E050E00E94C6413093F9
:1066F0007A03209379031092B3051092B2050091AA
:10670000C7071091C8072091C9073091CA07C60171
:1067100068E070E00E9491416F5F7F4FC50143E0E8
:10672000880F991F4A95E1F70E9491414B01AA24D5
:1067300097FCA094BA2C800E911EA21EB31E8092CC
:10674000C7079092C807A092C907B092CA07809164
:106750008F03482E5524C49CC001C59C900DD49C29
:10676000900D112460E270E00E9491413201661A9E
:10677000770A77FC7AC0E114F10409F06EC08091C9
:106780008605909187052091840530918505820FBB
:10679000931F68E070E00E9491416B0140E450E07B
:1067A000C40ED51E8091790390917A03AA2797FD94
:1067B000A095BA2F0CE1E02E02E0F02E012D112D54
:1067C000E81AF90A0A0B1B0BC501B4012EE036E0EA
:1067D00040E050E00E94C641E20EF31E041F151F68
:1067E000C801B70128E631E040E050E00E94C64110
:1067F000645B7040669DC001679D900D769D900D15
:106800001124B6010E9491419201220F331F240DE1
:10681000351D2617370734F0309521953F4F621705
:1068200073070CF4B9019B01442737FD4095542FA1
:1068300080914B0590914C05A0914D05B0914E056E
:10684000820F931FA41FB51F80934B0590934C0597
:10685000A0934D05B0934E050EC00894E108F108D1
:10686000F0927C03E0927B0306C084EF91E090936A
:106870007C0380937B038091B40581508093B405A1
:106880008F3F09F0B4C088E18093B405E090EB0736
:10689000FF2400E010E060912705709128058091A9
:1068A000290590912A05A80197010E94C6413093BD
:1068B00089062093880660912F057091300580919C
:1068C000310590913205A80197010E94C64130938D
:1068D0008B0620938A068091AB079091AC0790932A
:1068E0008D0680938C068091D0079091D10790936C
:1068F0008F0680938E068091C4079091C507909370
:1069000091068093900680918E0590918F059093CB
:106910009306809392066091570570915805809177
:10692000590590915A0520E032E040E050E00E9485
:10693000C641309395062093940680910E05909160
:106940000F05909399068093980680910C0390917F
:106950000D0390939B0680939A068091C60790E062
:1069600090939D0680939C068091BC0790E0909345
:106970009F0680939E068091CF0790E09093A1069A
:106980008093A0068091B10790E09093A306809336
:10699000A2068091D60790E09093A5068093A40666
:1069A0008091BD0790E09093A7068093A606809102
:1069B000BA079091BB079093A9068093A80680918F
:1069C000E2049091E3049093B1068093B006809125
:1069D0008005909181059093C5068093C4068091AF
:1069E0008205909183059093C7068093C606809197
:1069F0009605C090CD07D090CE07882391F0B601C0
:106A0000882777FD8095982F0E9437402091D207E4
:106A10003091D3074091D4075091D5070E94EF40A1
:106A20002DC06091270570912805809129059091CE
:106A30002A050E9437402091BE073091BF07409140
:106A4000C0075091C1070E94EF407B018C01B60145
:106A5000882777FD8095982F0E9437402091D20794
:106A60003091D3074091D4075091D5070E94EF4051
:106A70009B01AC01C801B7010E94383F0E9404404D
:106A80007093CE076093CD0780919705C090C207A1
:106A9000D090C307882391F0B601882777FD8095B1
:106AA000982F0E9437402091D2073091D307409110
:106AB000D4075091D5070E94EF402DC060912F055B
:106AC0007091300580913105909132050E943740D8
:106AD0002091BE073091BF074091C0075091C10778
:106AE0000E94EF407B018C01B601882777FD8095DD
:106AF000982F0E9437402091D2073091D3074091C0
:106B0000D4075091D5070E94EF409B01AC01C8010A
:106B1000B7010E94383F0E9404407093C3076093FE
:106B2000C2076091BE077091BF078091C007909126
:106B3000C10769837A838B839C836091C4077091BA
:106B4000C507882777FD8095982F0E9437407B01E5
:106B50008C016091D2077091D3078091D4079091F6
:106B6000D5079B01AC010E94383F9B01AC01C801D5
:106B7000B7010E94EF407B018C0160913705709155
:106B800038058091390590913A050E943740298156
:106B90003A814B815C810E94EF4020E030E040E090
:106BA0005FE30E94EF409B01AC01C801B7010E9466
:106BB000383F0E940440AB017093C5076093C4073F
:106BC0008091CD079091CE079093B3068093B20643
:106BD0002091C2073091C3073093B5062093B406C5
:106BE0008150904434F080E090E49093CE078093FD
:106BF000CD078091CD079091CE078050904C34F412
:106C000080E090EC9093CE078093CD0721503044E4
:106C100034F080E090E49093C3078093C2078091A2
:106C2000C2079091C3078050904C34F480E090EC00
:106C30009093C3078093C2074150504434F080E0E2
:106C400090E49093C5078093C4078091C407909106
:106C5000C5078050904C34F480E090EC9093C507C9
:106C60008093C4076B887C88660C771C660C771C45
:106C70008091DF07282F80FFC6C08091670584FDC3
:106C8000C2C080918C0321FF0EC0823310F5809129
:106C90008E0590918F054497909391058093900570
:106CA0001092B70519C02091850330918603280FF3
:106CB000311D8091E40790E0AC01249FC001259F25
:106CC000900D349F900D11244497909391058093DB
:106CD000900581E08093B70520918E0530918F0556
:106CE0004091900550919105421753070CF08BC0CD
:106CF0008091B705882309F486C080918D0390E0C8
:106D0000241B350BBC01629FC001639F900D729FD5
:106D1000900D112464E070E00E9491415B01C090ED
:106D2000F604D090F7046091570570915805809152
:106D3000590590915A05E0908E03FF2400E010E081
:106D400020E830E040E050E00E94C641C801B701B1
:106D50000E94524120E230E040E050E00E94C641F3
:106D60007EEF283E370714F428EE3EEF8091B505FC
:106D70009091B605FC01A4E0EE0FFF1FAA95E1F784
:106D8000E81BF90BC60162E070E00E949141E61B2E
:106D9000F70B81E02931380714F028E131E0E21BDC
:106DA000F30BC3018A199B098E0F9F1F60E170E0EE
:106DB0000E9491417093B6056093B5058091E007FC
:106DC00090E0880F991F880F991F6817790764F45E
:106DD000681679062CF09093B6058093B50504C02B
:106DE0007092B6056092B5058091B5059091B60593
:106DF0006816790624F47092B6056092B505609025
:106E0000B5057090B6058091EA07882E9924840113
:106E1000000F111F000F111FC801805590408615EB
:106E200097050CF43C01709297066092960680914B
:106E3000C5059091C605A091C705B091C80552E05F
:106E4000880F991FAA1FBB1F5A95D1F72091C4071D
:106E50003091C507281B390B91EA69167104ACF013
:106E6000F301F595E7952E173F070CF4F901C301DF
:106E700062E070E00E949141709561957F4FCF0173
:106E8000E617F7076CF4CB010BC0C901205B3F4F3D
:106E900014F480EB9FEF8135910514F080E590E0CC
:106EA000980126193709281739070CF4C9019301ED
:106EB000201B310B1C01821793070CF41901409021
:106EC000780550907905E091CD07F091CE07E4194F
:106ED000F509FC8FEB8FF093B907E093B80720E03A
:106EE00030E040E050E069817A818B819C810E9492
:106EF00072408823E1F16091CD057091CE058091BB
:106F0000CF059091D0050E9437405B016C016091E4
:106F10002705709128058091290590912A050E94E6
:106F2000374029813A814B815C810E94EF407B018F
:106F30008C01B201882777FD8095982F0E943740F9
:106F40009B01AC01C801B7010E94373F9B01AC0116
:106F5000C601B5010E94383F0E9404406093CD05F0
:106F60007093CE058093CF059093D0051BC06B8D99
:106F70007C8D9B01442737FD4095542F8091CD0592
:106F80009091CE05A091CF05B091D005820F931FAF
:106F9000A41FB51F8093CD059093CE05A093CF0578
:106FA000B093D0058091CD059091CE05A091CF05ED
:106FB000B091D00581509A4FA040B04064F080E07D
:106FC0009AEFA0E0B0E08093CD059093CE05A0931A
:106FD000CF05B093D0058091CD059091CE05A091BD
:106FE000CF05B091D00580509640AF4FBF4F64F4AD
:106FF00080E096E0AFEFBFEF8093CD059093CE0594
:10700000A093CF05B093D0052091870330918803DA
:107010004091890350918A032F8B388F498F5A8F63
:107020004091CD055091CE056091CF057091D0056E
:1070300049875A876B877C87C10137FE04C0882740
:1070400099278219930962E070E00E949141660DD0
:10705000771D882777FD8095982F2091A00330E039
:1070600040E050E00E94524120E430E040E050E037
:107070000E94C6413E872D87B901709561957F4F6B
:107080007E8B6D8B40907A0550907B058091C20776
:107090009091C307841995099CAB8BAB9093B30770
:1070A0008093B20720E030E040E050E069817A81CF
:1070B0008B819C810E9472408823E1F16091C90517
:1070C0007091CA058091CB059091CC050E94374004
:1070D0005B016C0160912F05709130058091310545
:1070E000909132050E94374029813A814B815C8121
:1070F0000E94EF407B018C01B201882777FD8095CB
:10710000982F0E9437409B01AC01C801B7010E9433
:10711000373F9B01AC01C601B5010E94383F0E9478
:1071200004406093C9057093CA058093CB05909382
:10713000CC051BC0ABA9BCA99D01442737FD4095D8
:10714000542F8091C9059091CA05A091CB05B091AB
:10715000CC05820F931FA41FB51F8093C905909380
:10716000CA05A093CB05B093CC058091C905909139
:10717000CA05A091CB05B091CC0581509A4FA04093
:10718000B04064F080E09AEFA0E0B0E08093C905E1
:107190009093CA05A093CB05B093CC058091C90507
:1071A0009091CA05A091CB05B091CC058050964036
:1071B000AF4FBF4F64F480E096E0AFEFBFEF809336
:1071C000C9059093CA05A093CB05B093CC052BA914
:1071D0003CA9B901882777FD8095982F0E943740F8
:1071E0007B018C016091C9057091CA058091CB0526
:1071F0009091CC050E9437409B01AC016F89788D3E
:10720000898D9A8D0E94EF409B01AC01C801B701A6
:107210000E94383F0E940440CD84DE846C157D05B9
:107220000CF46B014B8D5C8DBA01882777FD80953E
:10723000982F0E9437407B018C0169857A858B8568
:107240009C850E9437409B01AC016F89788D898DA8
:107250009A8D0E94EF409B01AC01C801B7010E94CA
:10726000383F0E9404402D853E85621773070CF459
:107270009B018D899E89821793070CF4C901880FA1
:10728000991F880F991F67E070E00E9491417B0170
:10729000C6016D897E89C616D7060CF4CB0163E062
:1072A00070E00E9491416B019701260D371DCB01C3
:1072B00062E070E00E949141FB018B010219130909
:1072C000C801820F931F64E070E00E94914186160E
:1072D000970614F4B40107C08091E90790E068179D
:1072E00079070CF4BC016093C6072E1B3F0BC90144
:1072F000820D931D64E070E00E949141861697060E
:1073000014F4B40107C08091E90790E06817790789
:107310000CF4BC016093BC0793012E193F09C8010E
:10732000820F931F64E070E00E94914186169706D9
:1073300014F4B40107C08091E90790E06817790759
:107340000CF4BC016093CF072E1B3F0BC901820DCB
:10735000931D64E070E00E9491418616970614F434
:10736000B40107C08091E90790E0681779070CF431
:10737000BC016093B107C101860D971D8C0D9D1D49
:1073800064E070E00E9491418616970614F4B401FF
:1073900007C08091E90790E0681779070CF4BC01F9
:1073A0006093D6076C187D08C3018219930964E0C5
:1073B00070E00E9491418616970644F08091E9079B
:1073C00090E04B01681779070CF44C018092BD07DF
:1073D000E4960FB6F894DEBF0FBECDBFDF91CF911C
:1073E0001F910F91FF90EF90DF90CF90BF90AF90E3
:1073F0009F908F907F906F905F904F903F902F90D5
:107400000895A0E0B0E0A80FB11D0E941842802DA1
:1074100090E00895A0E0B0E0A80FB11D062E0E94F4
:107420002A420895A0E0B0E0A80FB11D0E942542B5
:10743000CF010895A0E0B0E0A80FB11D0B010E949C
:1074400036420895863008F085E0A2E0B0E0082ECC
:107450000E942A420895982F863008F095E083E52F
:10746000989FD0011124AC59BF4FE7EDF7E0182EDB
:107470000E943B42A2E0B0E0092E0E942A420E94F4
:1074800091160895982F863008F095E083E5989F2F
:10749000D0011124AC59BF4FE7EDF7E0182E0E9440
:1074A00020420E949116089581E08093D70782E0E0
:1074B0008093D80793E09093D907E4E0E093DA074C
:1074C00055E05093DB0776E07093DC0787E080930C
:1074D000DD0768E06093DE0788EE8093DF073EE11A
:1074E0003093E0078BEF8093E2078AE08093E30715
:1074F0003093E1073093E5079093E4076093E60744
:1075000090E19093E7077093E8076093E90786EEB0
:107510008093EA073093EB0780E88093EC0744E61A
:107520004093ED0788E78093EE078EE58093EF07A1
:1075300083E28093F00784E18093F1071092F207D1
:107540009093F3071092F4071092F5071092F60744
:107550001092F70710920708109208081092090875
:1075600010920A084093F80788E28093F907109276
:10757000190892E39093FA0786E98093FB075093EA
:10758000FC079093FD072AE52093FE079093FF07E1
:1075900010921808209300085093010885E5809305
:1075A00002088093030880E280930408E0930508B2
:1075B000909306088FE580930B0883EF80930D0866
:1075C00030930C0830930E088DEF80930F08409392
:1075D000100820931108209312082093130810928A
:1075E00014087093150860931608AEE1B8E0EBEA52
:1075F000F3E089E001900D928150E1F7089581E078
:107600008093D70782E08093D80723E02093D9079F
:10761000E4E0E093DA0735E03093DB0766E060935F
:10762000DC0787E08093DD0758E05093DE0788E6AB
:107630008093DF079EE19093E0078BEF8093E20752
:107640008AE08093E3079093E1079093E507209306
:10765000E4078CE08093E60780E18093E70760937E
:10766000E8075093E90786EE8093EA079093EB07CB
:1076700080E88093EC0780E58093ED0788E78093AE
:10768000EE078EE58093EF0783E28093F0079093F7
:10769000F1071092F20740E24093F3071092F407CB
:1076A0001092F5071092F6071092F707109207084C
:1076B000109208081092090810920A0874E6709354
:1076C000F80788E28093F9071092190892E39093E3
:1076D000FA0786E98093FB073093FC079093FD0738
:1076E0002AE52093FE079093FF0710921808209335
:1076F00000083093010885E5809302088093030811
:1077000040930408E09305088BE4809306088FE516
:1077100080930B0883EF80930D0884E180930C081D
:1077200080930E088DEF80930F08709310082093BC
:1077300011082093120820931308109214086093E4
:10774000150850931608AEE1B8E0E5EBF3E087E0EA
:1077500001900D928150E1F7089581E08093D70761
:1077600082E08093D80783E08093D90764E0609338
:10777000DA0745E04093DB07E6E0E093DC0787E0CB
:107780008093DD0778E07093DE0788E68093DF075B
:107790009EE19093E0078BEF8093E2078AE080936D
:1077A000E3079093E1079093E5076093E4073FE0D8
:1077B0003093E6079093E7078CE08093E807709397
:1077C000E90786EE8093EA079093EB0780E88093C1
:1077D000EC0780E58093ED0756E95093EE078EE5C0
:1077E0008093EF0783E28093F0079093F107109264
:1077F000F20780E28093F3071092F4071092F507E6
:107800001092F6071092F7071092070810920808D6
:107810001092090810920A0824E62093F80788E2DB
:107820008093F9071092190882E38093FA07509326
:10783000FB074093FC078093FD079AE59093FE07B2
:107840008093FF0710921808909300084093010856
:1078500085E5809302088093030880E18093040803
:1078600060930508209306088FE580930B0883EF4B
:1078700080930D0830930C0830930E088DEF8093A1
:107880000F0820931008909311089093120890937A
:10789000130810921408E093150870931608AEE1CF
:1078A000B8E0EDEBF3E086E001900D928150E1F756
:1078B000089522E030E0D9010E941842802D8630E0
:1078C00028F082E0D901082E0E942A4290E0089513
:1078D0000F931F93CF93DF93A1E0B0E00E94184273
:1078E000802D873469F186E994E09F938F931F92EE
:1078F0000E947C080E94AD3BC0E0D0E00F900F904A
:107900000F900C2FC23039F0C33019F40E94543A52
:1079100004C0C43010F00E94FF3A802F0E942B3A1E
:107920002196C630D10569F7A2E0B0E083E0082EC9
:107930000E942A42A1E0B0E087E4082E0E942A4279
:1079400002E010E0D8010E941842802D0E94423AC5
:10795000D8010E941842802D90E09F938F938DE76D
:1079600094E09F938F931F920E947C080F900F903A
:107970000F900F900F90DF91CF911F910F9108956D
:10798000CF93DF93DC01EC01EA81FB8121918E81B1
:10799000815019F48981E81BF109ED01FB83EA8329
:1079A0008E839FB7F8948C9181508C939FBF822FC8
:1079B00090E0DF91CF910895FC011082758364837C
:1079C000738362834183478346830895CF93DF9314
:1079D000DC019C91ED018981981718F080E090E01E
:1079E00016C0ED01EC81FD8161938F81815019F406
:1079F0008981E81BF109ED018F83FD83EC839FB73B
:107A0000F8948C918F5F8C939FBF81E090E0DF9121
:107A1000CF910895FC0180818823E9F3CF010E9472
:107A2000C03C90E00895FC018081882319F48FEF19
:107A30009FEF0895CF010E94C03C90E008959FB74A
:107A4000F8948091C9008F778093C9008091C90014
:107A50008F7B8093C9008091C9008F7D8093C9007E
:107A60005A9A52985B9A539A1092CD008AE2809368
:107A7000CC008091C80082608093C80088E1809328
:107A8000C9008091CA008F778093CA008091CA0094
:107A90008F7B8093CA008091CA008F7D8093CA003B
:107AA0008091CA008F7E8093CA008091CA00877F30
:107AB0008093CA008091C9008B7F8093C900809118
:107AC000CA0084608093CA008091CA00826080935B
:107AD000CA0002C08091CE008091C80087FDFACF15
:107AE0008091C90080688093C9008091C90080643A
:107AF0008093C9009FBF08951F920F920FB60F92F7
:107B000011248F938091CE008F910F900FBE0F9014
:107B10001F901895A8E0B0E0E0E9FDE30C94EB417C
:107B20007B018C01611571058105910519F482E0D5
:107B300089835AC083E089838EE1C82ED12CDC82F0
:107B4000CB82ED82FE820F831887C801B7010E94A5
:107B5000FD3DBC016150704077FF33C0EE27FF2729
:107B6000E61BF70B20E030E040E050E081E090E0E1
:107B7000A0E0B0E00E2E04C0880F991FAA1FBB1F03
:107B80000A94D2F70197A109B1098E219F21A02360
:107B9000B1230097A105B10521F021E030E040E0DC
:107BA00050E004C016950795F794E794EA95D2F74C
:107BB0002E293F29402B512B2D833E834F835887FD
:107BC0000FC06115710581F0062E04C0EE0CFF1C7C
:107BD000001F111F0A94D2F7ED82FE820F831887CF
:107BE000C61AD70ADC82CB821A82CE0101960E9485
:107BF0004A3EE8E028960C940742EF92FF920F93DA
:107C00001F939B01AC01203080E0380781E04807DA
:107C100080E0580780F42F3F31054105510509F0F8
:107C200020F4EE24FF24870119C068E0E62EF12C31
:107C3000012D112D13C0203080E0380780E0480767
:107C400081E0580730F490E1E92EF12C012D112D3F
:107C500005C088E1E82EF12C012D112D80E290E085
:107C6000A0E0B0E08E199F09A00BB10B04C056959F
:107C7000479537952795EA94D2F7F901EC53FC4FD5
:107C80002081821B9109A109B1091F910F91FF90D9
:107C9000EF9008959F92AF92BF92CF92DF92EF92B2
:107CA000FF920F931F93EE24FF248701FC01248190
:107CB00035814681578191808081823010F4406106
:107CC000A2C0843009F49BC0823029F420E030E067
:107CD00040E050E005C0211531054105510519F47A
:107CE000E0E0F0E092C0828193816FEF82389607E6
:107CF0000CF05AC062E87FEF681B790B6A3171059E
:107D00002CF020E030E040E050E02AC0AA24BB2460
:107D1000650181E090E0A0E0B0E0062E04C0880F8D
:107D2000991FAA1FBB1F0A94D2F70197A109B10995
:107D300082239323A423B5230097A105B10529F03D
:107D400071E0A72EB12CC12CD12C04C056954795BB
:107D5000379527956A95D2F72A293B294C295D2921
:107D6000DA01C9018F779070A070B07080349105EE
:107D7000A105B10539F427FF09C0205C3F4F4F4FE3
:107D80005F4F04C0215C3F4F4F4F5F4F80E090E05A
:107D9000203060E0360760E0460760E4560710F0E8
:107DA00081E090E0FC0123C08038910544F5FC019E
:107DB000E158FF4FDA01C9018F779070A070B07061
:107DC00080349105A105B10539F427FF09C0205C75
:107DD0003F4F4F4F5F4F04C0215C3F4F4F4F5F4FAE
:107DE00057FF05C05695479537952795319687E0FB
:107DF00056954795379527958A95D1F706C020E087
:107E000030E040E050E0EFEFF0E0E22EF32E942F70
:107E10009F77802F8078892B9E2F9795992797950C
:107E20008F77082F092B9E2F9695812F8078892B8D
:107E30009794992497948F77182F1929C801B7011F
:107E40001F910F91FF90EF90DF90CF90BF90AF9078
:107E50009F900895FC014150504030F0019006166B
:107E6000D1F73197CF010895882799270895505861
:107E7000BB27AA270ED079C16AD130F06FD120F08C
:107E800031F49F3F11F41EF45FC10EF4E095E7FB5F
:107E900055C1E92F7BD180F3BA17620773078407B6
:107EA000950718F071F49EF593C10EF4E0950B2E32
:107EB000BA2FA02D0B01B90190010C01CA01A0013C
:107EC0001124FF27591B99F0593F50F4503E68F197
:107ED0001A16F040A22F232F342F4427585FF3CFD8
:107EE000469537952795A795F0405395C9F77EF4A9
:107EF0001F16BA0B620B730B840BBAF09150A1F0F2
:107F0000FF0FBB1F661F771F881FC2F70EC0BA0F77
:107F1000621F731F841F48F4879577956795B795FF
:107F2000F7959E3F08F0B3CF9395880F08F09927F7
:107F3000EE0F9795879508950CD017C10FD140F09B
:107F400006D130F021F45F3F19F0F8C0511141C162
:107F5000FBC01CD198F39923C9F35523B1F3951BAA
:107F6000550BBB27AA2762177307840738F09F5F5A
:107F70005F4F220F331F441FAA1FA9F333D00E2EC9
:107F80003AF0E0E830D091505040E695001CCAF736
:107F900029D0FE2F27D0660F771F881FBB1F2617FB
:107FA00037074807AB07B0E809F0BB0B802DBF01CE
:107FB000FF2793585F4F2AF09E3F510568F0BEC0DF
:107FC00008C15F3FECF3983EDCF3869577956795A3
:107FD000B795F7959F5FC9F7880F911D969587957F
:107FE00097F90895E1E0660F771F881FBB1F62179E
:107FF00073078407BA0720F0621B730B840BBA0B5C
:10800000EE1F88F7E095089504D06894B111E1C09F
:108010000895C4D088F09F5790F0B92F9927B75191
:10802000A0F0D1F0660F771F881F991F1AF0BA953C
:10803000C9F712C0B13081F0CBD0B1E00895C8C00B
:10804000672F782F8827B85F39F0B93FCCF3869532
:1080500077956795B395D9F73EF49095809570958F
:1080600061957F4F8F4F9F4F0895E89409C097FB0C
:108070003EF490958095709561957F4F8F4F9F4FFF
:108080009923A9F0F92F96E9BB279395F695879543
:1080900077956795B795F111F8CFFAF4BB0F11F406
:1080A00060FF1BC06F5F7F4F8F4F9F4F16C08823AD
:1080B00011F096E911C0772321F09EE8872F762FE3
:1080C00005C0662371F096E8862F70E060E02AF024
:1080D0009A95660F771F881FDAF7880F9695879510
:1080E00097F9089507D008F481E0089503D008F4C3
:1080F0008FEF0895990F0008550FAA0BE0E8FEEFE7
:1081000016161706E807F907C0F012161306E4075B
:10811000F50798F0621B730B840B950B39F40A2654
:1081200061F0232B242B252B21F408950A2609F432
:10813000A140A6958FEF811D811D089597F99F6736
:1081400080E870E060E008959FEF80EC08950024DF
:108150000A941616170618060906089500240A94AC
:1081600012161306140605060895092E0394000C32
:1081700011F4882352F0BB0F40F4BF2B11F460FFC1
:1081800004C06F5F7F4F8F4F9F4F089557FD9058EA
:10819000440F551F59F05F3F71F04795880F97FBCB
:1081A000991F61F09F3F79F0879508951216130685
:1081B0001406551FF2CF4695F1DF08C016161706B4
:1081C0001806991FF1CF86957105610508940895E9
:1081D000E894BB2766277727CB0197F908950BD042
:1081E000C4CFB5DF28F0BADF18F0952309F0A6CF89
:1081F000ABCF1124EECFCADFA0F3959FD1F3950F3B
:1082000050E0551F629FF001729FBB27F00DB11D1A
:10821000639FAA27F00DB11DAA1F649F6627B00DAA
:10822000A11D661F829F2227B00DA11D621F739F93
:10823000B00DA11D621F839FA00D611D221F749FA1
:108240003327A00D611D231F849F600D211D822FE8
:10825000762F6A2F11249F5750408AF0E1F088232F
:108260004AF0EE0FFF1FBB1F661F771F881F91503C
:108270005040A9F79E3F510570F060CFAACF5F3FF5
:10828000ECF3983EDCF3869577956795B795F7956F
:10829000E7959F5FC1F7FE2B880F911D96958795F7
:1082A00097F90895629FD001739FF001829FE00DBE
:1082B000F11D649FE00DF11D929FF00D839FF00D65
:1082C000749FF00D659FF00D9927729FB00DE11D11
:1082D000F91F639FB00DE11DF91FBD01CF011124EE
:1082E0000895991B79E004C0991F961708F0961B12
:1082F000881F7A95C9F780950895AA1BBB1B51E189
:1083000007C0AA1FBB1FA617B70710F0A61BB70B05
:10831000881F991F5A95A9F780959095BC01CD01AA
:10832000089597FB092E07260AD077FD04D0E5DFD4
:1083300006D000201AF4709561957F4F0895F6F7E6
:10834000909581959F4F0895A1E21A2EAA1BBB1B01
:10835000FD010DC0AA1FBB1FEE1FFF1FA217B30711
:10836000E407F50720F0A21BB30BE40BF50B661F27
:10837000771F881F991F1A9469F7609570958095EB
:1083800090959B01AC01BD01CF01089597FB092E8B
:1083900005260ED057FD04D0D7DF0AD0001C38F4D4
:1083A00050954095309521953F4F4F4F5F4F089521
:1083B000F6F790958095709561957F4F8F4F9F4F01
:1083C00008952F923F924F925F926F927F928F9279
:1083D0009F92AF92BF92CF92DF92EF92FF920F9354
:1083E0001F93CF93DF93CDB7DEB7CA1BDB0B0FB65E
:1083F000F894DEBF0FBECDBF09942A88398848881B
:108400005F846E847D848C849B84AA84B984C884B0
:10841000DF80EE80FD800C811B81AA81B981CE0FA7
:10842000D11D0FB6F894DEBF0FBECDBFED0108958C
:10843000F999FECFB2BDA1BDF89A119600B4089586
:10844000F7DF01921A94E1F70895F2DFE02DF0DFF3
:10845000F02D0895F999FECFB2BDA1BD00BC1196D3
:108460000FB6F894FA9AF99A0FBE0895F3DF012C2B
:10847000F1DF112408950190EDDF1A94E1F70895DA
:02848000FFCF2C
:108482000AFF0164496E74656772616C4E69636BC1
:1084920020202020496E74656772616C526F6C6C8B
:1084A200202020204163634E69636B20202020201E
:1084B20020202020416363526F6C6C2020202020FA
:1084C200202020204779726F5961772020202020B8
:1084D2002020202052656164696E6748656967687B
:1084E200742020204163635A202020202020202055
:1084F20020202020476173202020202020202020BF
:10850200202020205265636569766572204C65766D
:10851200656C2020566F6C746167652020202020D6
:10852200202020204D6F746F722046726F6E744C43
:10853200656674204D6F746F722046726F6E74524E
:10854200696768744D6F746F7220526561724C6511
:10855200667420204D6F746F722052656172526989
:10856200676874204D6F746F722052696768742057
:10857200202020204D6F746F72204C65667420207D
:10858200202020204163635F5A20202020202020C9
:1085920020202020535049204572726F72202020E3
:1085A20020202020535049204F6B202020202020C3
:1085B20020202020202020202020202020202020B9
:1085C20020202020536572766F202020202020203A
:1085D200202020204E69636B202020202020202094
:1085E20020202020526F6C6C202020202020202070
:1085F2002020202020202020202020202020202079
:108602002020202020202020202020202020202068
:108612002020202020202020202020202020202058
:108622002020202020202020202020202020202048
:108632002020202020202020202020202020202038
:108642002020202020202020202020202020202028
:108652002020202020202020202020202020202018
:10866200202020204750535F4E69636B202020203A
:10867200202020204750535F526F6C6C2020202016
:1086820020202020FFFF0128006400806400737313
:1086920073007D0000FF03010203040506070809B9
:1086A2000A48656C6C6F20576F726C6400000000A2
:1086B20000000000000000000000000000000000B8
:1086C20000000000000000000000000000000000A8
:1086D2000000000000000000000000000000000098
:1086E2000000000000000000000000000000000088
:1086F200000B0101640001FFFFFFFFF40190D003B2
:108702000090D00300ECFF17B7D13830FB103A408D
:108712009696020A00000000000000006446000075
:108722006400000000000000000001426567696EFD
:108732006E657200004E6F726D616C000053706F57
:108742007274000000010202030303030404040420
:1087520004040404050505050505050505050505CB
:1087620005050505060606060606060606060606AB
:108772000606060606060606060606060606060697
:10878200060606060707070707070707070707077B
:108792000707070707070707070707070707070767
:1087A2000707070707070707070707070707070757
:1087B2000707070707070707070707070707070747
:1087C200070707070808080808080808080808082B
:1087D2000808080808080808080808080808080817
:1087E2000808080808080808080808080808080807
:1087F20008080808080808080808080808080808F7
:1088020008080808080808080808080808080808E6
:1088120008080808080808080808080808080808D6
:1088220008080808080808080808080808080808C6
:1088320008080808080808080808080808080808B6
:048842000808080812
:00000001FF
